:100000000C941E1B0C94451B0C94451B0C94451B17
:100010000C94451B0C94592C0C94451B0C94451BBB
:100020000C94451B0C94451B0C94451B0C94B41D5F
:100030000C94451B0C94451B0C94451B0C94451BC0
:100040000C94451B0C94451B0C94451B0C94451BB0
:100050000C94451B0C945A2C0C94451B0C94451B7A
:100060000C94451B0C94451B0000E0FF10841F00FE
:10007000228A10806636FF070F044A616E7561722E
:100080000046656272756172004DC3A4727A0041C8
:100090007072696C004D6169004A756E69004A753D
:1000A0006C69004175677573740053657074656D94
:1000B000626572004F6B746F626572004E6F766599
:1000C0006D6265720044657A656D626572004DC34C
:1000D000BC6C6C6B616C656E6465720000001FF82F
:1000E00000F8E0071F00E0FF20253032643A253099
:1000F00032643A253032642000536F6E6E7461674B
:10010000004D6F6E746167004469656E737461675A
:10011000004D697474776F636800446F6E6E65722A
:1001200073746167004672656974616700536F6E2E
:100130006E6162656E64002025642E2025532025A3
:10014000642530326420002025532000E0FF0000A9
:100150000000FFFFFFFFFFFF0000FFFFFFFF4B65F9
:10016000696E20416266616C6C00427261756E65F9
:1001700020546F6E6E6500426C61756520546F6E21
:100180006E6500477261756520546F6E6E6500473D
:10019000656C626520546F6E6E6500686575746588
:1001A000006D6F7267656E00C3BC6265726D6F72C1
:1001B00067656E00AC2020001A2092011E202620C8
:1001C00020202120C6023020600139205201200069
:1001D0007D0120002000182019201C201D20222035
:1001E00013201420DC02222161013A205301200057
:1001F0007E017801000003F0A5A503FCA5A5012957
:10020000000DFA0A040C1925332D27221E1A000DA1
:10021000FB0C04191E2023183D25190B00000AF6BB
:1002200001010700010C030C030DF5002E40000036
:100230000100000D0D000015F4070000002264010C
:10024000022A4D062A000600000000000002F30109
:100250000003F05A5A03FC5A5A0CFD000010141205
:100260000004484016160135023648023A5512F28B
:10027000285B7F0808000015480407010000630898
:100280000805F70100100004F833000000FC1320FB
:10029000E00054C5081152100055555555552255CA
:1002A000657C88788608859688877886B877151063
:1002B00055515656620650A06666526195652520D6
:1002C000551550C455E1171C15014024C5C1151B17
:1002D00075005555508152155852115105115299BA
:1002E000697777778C77770011888888588888783D
:1002F000675555555A5555001166666656666666C9
:100300006600000000000000000000000000000087
:1003100000000000000000000000000000000000DD
:1003200000000000000000000000000000000000CD
:1003300000000000000000000000000000000000BD
:1003400000000000000000000000000000000000AD
:10035000000000000000000000000000000000009D
:10036000000000000000000000000000000000008D
:10037000000000000000001F00000000F800000066
:100380000000000000000000000000000036000037
:10039000000000000000000000000000000000005D
:1003A0000000000000000000000000000000E00E5F
:1003B0000380E81B01E00000000380380E03639D0A
:1003C000DB0000E80E00700700E80D800000070069
:1003D0003803806C070000000000000000000000EF
:1003E000000000000000000000000000000000000D
:1003F00000000000000000000000000000000000FD
:1004000000000000000000000000000000000000EC
:1004100000000000000000000000000000000000DC
:1004200000000000000000000000000000000000CC
:1004300000000000000000000000000000000000BC
:1004400000000000000000000000000000000000AC
:10045000000000000000000000000000000000009C
:10046000000000000000000000000000000000008C
:10047000000001C00000000E0000000000000000AD
:10048000000000000000000006C0000000000000A6
:100490000000000000000000FF80000000000000DD
:1004A0000000000000000000000C0180F81703604D
:1004B0003C00000000300603E06C337F6000170052
:1004C000C00C01F01701B0000000600600F80D80BC
:1004D000C000000000000000000F0000000000004D
:1004E000000000000000000000000000000000000C
:1004F00000000000000000000000001000000000EC
:1005000000000000000000000000000000000000EB
:1005100000000000000000000000000000000000DB
:1005200000000000000000000000000000000000CB
:1005300000000000000000000000000000000000BB
:1005400000000000000000000000000000000000AB
:10055000000000000000000000000000000000009B
:10056000000000000000000000000000000000008B
:10057000000000000000000000000000000000007B
:10058000000000000000000000000000000000006B
:100590000000001FF000000000000000000000004C
:1005A00000000000000000000000000780000000C4
:1005B000000000000000000000000000000000003B
:1005C0000000000004000000000000000000000027
:1005D0000000000001E0000000000000000000003A
:1005E000000000000000000000000000000000000B
:1005F00000000003330D8F8F0E03E0C7E100000001
:100600003BF030FC7E071F87CFF3F1F000000000C5
:1006100000FC07F80E0FF03F8FF0FF9FE1FC6066D3
:1006200003307300F1E7061F87F83F0FF87F3FF6AE
:1006300006C06E38FE1F03BFDF9E3C00380060001E
:10064000003001F001806660300000000000000012
:1006500000180000000000000007B7800000F8004C
:100660000F00000018061DF3801FC00FFF81FE0061
:10067000331B3600000000EBEC61F00000007CC092
:10068000E000C3E0039CC7CD8FC7C0000007E001B6
:10069000F003FF7001FE0073E0071C38E3E3000085
:1006A000700E01C0380700F03FFC3F8FF9FF3FE7B5
:1006B000FCCCC63FC3830FC0FC0FC0FC0FC0007F43
:1006C000D81981981981B03B003E0701C1C1D0D82B
:1006D0003C000000381C0E0D9CEED8F83A0701C013
:1006E000703A0D800000700E0381B038600D806696
:1006F00063F3FBF1C0FE18FCF80000077E0E3FDF3D
:10070000E0E7F1FDFEFF7F00000000003FC1FF8336
:10071000E1FF0FF9FF1FF3FC7FCC0CC0661C601ECD
:100720003CF0C7F8FF8FF1FF9FF7FEC0DC1DCF9DA7
:10073000C770E7FBFBC78003000C000006003E000B
:10074000300CCC0600000000000000000300000098
:100750000000000000F6F000FE3F7C03E000000314
:1007600000C7FEE007FC03FFFFBFFFF66366C000A3
:1007700000001711DC1C000007C71C380018FE0021
:100780007398FDB79EF8000003CF0036187FEC0089
:100790007FC01E7C01E30F387CE0001F03E07C0F6C
:1007A00081F03E07FF8FF9FF3FE7FCFF9998C7FCF8
:1007B0007863FC3FC3FC3FC3FC001FF303303303EB
:1007C00030370E600FE060307C2E1B078000000386
:1007D0000303E1B19BFB1E05C060301F05C1B000E3
:1007E00000060180F836060C01B00CCC7E7F6670E6
:1007F0001DC339CE0C0000FCE7C73B9C3CE07B816D
:10080000DCEE700001801807B87CF87C30E3CF3054
:10081000F300601E7981980CC70C03C79E19E798F6
:1008200073CF30739E0C181B83B9F39DC7380E67C6
:1008300019F8000001800000C0060006000180C019
:100840000000000000000000600000000000000048
:100850001CCE0018CF6D8070000000601806DC0010
:10086000E780F781B076F684484800000000023B3C
:1008700080000000D801CE00031DC826631F80C081
:10088000CF00000060600443039C000FB000CD80E7
:100890000CE06703980003E07C0F81F03E07C0F88E
:1008A00003CF300600C018033318C3CF0CF3CF3C7E
:1008B000F3CF3CF3C0079E606606606606738FF157
:1008C000DC0000000000000000000000000000004C
:1008D0000007E0000000000000000C0040000000E5
:1008E000000001800001999FCD0CCE03B8673BE169
:1008F00080001F9CF8C303879C0E00730D8630C0D8
:10090000F7FBC0E31DFF8D860C70E60E600C0387BD
:1009100030330199C18078F3E338730670E60671CD
:10092000C1830338E3BE63F8E701CCE33F00003F37
:100930003F87E3F8F9F1FCDE3333D9FBE7F0FC7FC6
:100940000FE7CF9F61B8FCE7E3E0CFE318C00319DE
:10095000C1B00E0000000C1FE0DF001C701C7036E0
:100960000EDED98D9B000000000045D0F803FF9BF0
:100970007F39C067E33BFEFC63C033CFE007F81B61
:10098000E600D860F1818DF60019B001980DC037EE
:1009900000C06C0D81B03606C0D83B0070E600C0C8
:1009A00018030066631839F19C39C39C39C39C3B1A
:1009B00098E3CC0CC0CC0CC0CE71FF3387E3F1F8C8
:1009C000FC7E3F1FF87E3E1F0F87C66630FC7F0F00
:1009D000C3F0FC3F0FC181FCC330CC330D833F9883
:1009E000303003F9E1FB807F00E700300003E19B3A
:1009F00000E1F1F3F9FC1C73B0C6187EFF7E00E73E
:100A0000FFF3B8C38E00C1CC018070060660337856
:100A1000300FBE6C670E61CE1CC3CF803060671C88
:100A200077DC3E0FC0719C6E70000FE7F9FCFF3F52
:100A3000BE7F9FE666F33FFCFF3FCFF3FCFBFBEC82
:100A4000331BBEEEEE39FC631800637F3607E0000F
:100A5000000FF3FC1FE003E0730606C39BDB31B31A
:100A600063E000000008BA3F9CFFFB6FE3F00DFE5F
:100A7000703F9F8C7C06CDFC7EFF034CC01F7FBD6A
:100A8000F031BEC0033EFC3701B83EC0181DC3B8EC
:100A9000770EE1DC3B87600E00C0180300600CCCD1
:100AA00063073633873873873873877F9CF981985B
:100AB00019819818FC30E671FCFE7F3F9FCFE7FF5D
:100AC0009FCFE7F3F9FCCCC63FCFF3FCFF3FCFF35A
:100AD000FC007F1866198661B8E7FB8E06003F3F71
:100AE0001EE00FC01CE03FC0006C30601C3E767FF3
:100AF000BFC38FE738003F0003F03CFEF6771FF1DD
:100B0000801819FF3F8C00FFCC067F0601F7CDCC83
:100B1000C0CFF9819FF8FE060C0C670EDB8380F0D6
:100B20001C338DCE0001DCE73B9CE7730E73DCCCFD
:100B3000FC677B9EE739CE739D7731867777DCF94A
:100B4000C7039C639F6C6606C0FC000001FE0C039B
:100B5000F8003F8E60FFD8E37B0000007C000000BF
:100B6000011747739CF76C1C3C003BDF8771E19FCA
:100B7000C0901F8FC0604988000FF7FE0633D80071
:100B800067DF86E03607F80003B8770EE1DC3B87C5
:100B900071CFF9801FF3FE7FCFF9998CFC66E66078
:100BA00066066066066067E33B3033033033030F4D
:100BB000060CCC3B9DCEE773B9DCEF73B9DCEE7766
:100BC0003B9998C739EE739CE739CE73BFCEF30CCF
:100BD000C330CC371CE771C0C006C3F01DE3FB0374
:100BE0000C07F8001D860C0F01CCCE773871FEFF84
:100BF000000783FC1E0F1F8EDC73FF3003033FE7EB
:100C0000F18F9FF980CFF0C036D99D9819FE30330F
:100C1000FE0FE0C1818EE0FBF0701E038631800084
:100C2000000F9CE6039CFE61CE71999F0CC7338C2C
:100C3000E739CE738F8630CEE6FB1F1DC0E78C7B75
:100C4000FD8DFCD80E00000006018007FBE3FB8C45
:100C50001FFB1C6F6000000F800000000000F83BCD
:100C60009FED87078037C3F0C6FF03BC120203F075
:100C70000C09F10000300000C61B300001F839C13A
:100C8000FE067060E39C738E71CE39C739FF300366
:100C9000FE7FCFF9FF33318C0CCECC0CC0CC0CC016
:100CA000CC0C786E66066066066061E0C199C1F0A2
:100CB000F87C3E1F0F87FE603F9FCFE7F33318E7B6
:100CC00038CE739CE739CE77F9FE6198661986773E
:100CD0001CE7701801FC1E077E77E061801803C3D3
:100CE000B0C183C01B9806C31C39CFE000FC7F8FC6
:100CF000C1C363FBFE61E70060E600C039F3033067
:100D000019CE1806FB31B30330060667803C183055
:100D100031DC1F7C1F0180E0C730000007F30CC0EE
:100D2000619FCC30CC3333F198C6619866198661E7
:100D3000FCC618F8FFE1C3B838F18F4FB1BC1B01F6
:100D4000C0000000C03000DF7C0F71C703670DECEE
:100D5000000001FFFFFFF800001FC761FDB1C06088
:100D600006D8181DC300638366C07E019FA660007D
:100D700006000018C36600003F07383FC1CE1C1FA5
:100D8000F3FE7FCFF9FF3FEFF00700600C018030EA
:100D90000666318398D9819819819819819F8F9C13
:100DA000C0CC0CC0CC0C1818733CFE7F3F9FCFE723
:100DB000F3FFCC07F3F9FCFE6663186619866198A9
:100DC0006619860036CC330CC330CEE30CEE03003C
:100DD0003F9AC0ECCC7C0C30030078773830F0E3DD
:100DE0007FB8D86386181C0007E007E0306C7F7F6F
:100DF000CC0CE1CC1CC01807066066C330E300DFF2
:100E0000663E70E600EDCC78E183070E1F03EF87A6
:100E1000F0303818E6000000FE73980E7301873931
:100E200086667E3318CC339CE739CC0F98C71F1FDA
:100E30007C7C7E0E0E31C0063383603800000018C3
:100E400006003B6DB86E38E06DC1BD8000003FFF0D
:100E5000FFFF000000F8EE7036700C00DFE703FBC8
:100E6000FC0F7067980FC033F4CC0000C0000398EB
:100E70006C000007E1CF0E3833C783FE7FCFF9FF48
:100E80003FE7FDFE00E1CC0180300600CCC63073A8
:100E90001F3873873873873877F9E39C39C39C39D7
:100EA000C38303FE639FCFE7F3F9FCFE7B0180C0A1
:100EB0006030180CCC639CC339CE739CE739C307F0
:100EC000F98E6398E639F8739F800007E3F8399943
:100ED000CF81CE0060000EE7061C1CEFF73BDC70F4
:100EE000E77780003C00F0000DDFDC1D839E7987F2
:100EF000980300F3CC0CDDE61C6019CCC3CF3CC0DA
:100F00001FF9879E7060F3C3E07DF0EE0607031CB7
:100F1000C000001DCE73B9CE7730E730CCCCE6638D
:100F20001986739CE77987731DE3E3EF8F87C3808E
:100F3000C63000C67B6C070000000300C0076DB719
:100F40009CE7BC0DB837B0000000000000000000B6
:100F50007739CF76DC01801BDDFBFF8C19FE06069E
:100F600000FC0003030000000000770D800001F882
:100F70003B61CF0ED9E0E0FC1F83F07E0FC1F8C0CB
:100F80001E7980300600C01998C61E61E79E79E779
:100F90009E79E79EE73CF3CF3CF3CF3CF0607F8D3A
:100FA000F3B9DCEE773B9DCEF73B9DCEE773B99965
:100FB0008C73986739CE739CE73860F73BCEF3BCEF
:100FC000EF1F0E71F00C00FC7F0E3F3FF839C000A0
:100FD000180DCFC0C7FBFC0CFF3F8C1FEFE1860153
:100FE000801800C1FFFB83BFF1FF3FE3FE600FF9F4
:100FF000819BFCC1CFF3399878FF1801FE3073FE56
:101000000C1FF838071C38E0C1FF6398000003FD8F
:10101000FE7F3FCFE61FE619999CCC6330CFF3FCEF
:10102000FF30FE7BFC383DE3B8F87F18C60018C7D8
:10103000EDB0C1B18C6060FF01CFBEFF9C7FFFBFF0
:10104000FEF60000000000000000000FE73FFEDB9E
:10105000F830037FBFE821830F8073801F80003941
:10106000C0001FE0000FE1B000003F0E7E73C19F83
:10107000B81C1F83F07E0FC1F83E1FF1FF3FE7FC55
:10108000FF9FF33318FF8C3C7F87F87F87F87F80C2
:1010900007FC7FE7FE7FE7FE0C0C01BE7FBFDFEFA2
:1010A000F7FBFDFFE7F3F9FCFE7F33318FF30CFF15
:1010B0003FCFF3FCFF001FE7F9FE7F9FE3E1FE3E19
:1010C00001801F87C1C3C3F60738000301B1F818B8
:1010D000FF3F018FC3E181F8F830C0000000183BEA
:1010E000FE7077FC1FC7F87FCC00FC30333F181D23
:1010F000FE6733070FC3001FE60F3F8181FE070025
:10110000E38E1E183FEC730000003FBF87C3F8F862
:10111000C1ECC33331D98C6618FC7F0FE60F8F3FCB
:1011200087071CE38E0FE318C003F87DF6383631CD
:101130008C0C1FE039F7CFE007FFFFFFFFC0000076
:1011400000000000000000F803FF9F7F060067E634
:101150007C003060F007E000000003F00003FC00BA
:1011600001FC3600000001C18E7C70663B83F07E7E
:101170000FC1F83F07C3FE1FC7FCFF9FF3FE666366
:101180001FE18387E07E07E07E07E001FF07F87F2D
:1011900087F87F8181803387F3F9FCFE7F3FBEF8BB
:1011A0007C3E1F0F87C66630FC618FC3F0FC3F0F8B
:1011B000C003F87F1FC7F1FC383F83800000002088
:1011C00000000000E7000020000000000000000018
:1011D0000000000000080000000003807000000014
:1011E00000000000000000000000000000000000FF
:1011F0000000000C000000000000000000000000E3
:10120000018060000000000000000000738000E02A
:1012100000000000000C000C0000000000000003B3
:10122000C0007338000000004702400001806000E9
:1012300000000000000000000000000000000000AE
:101240000000000000000000000CC00000000CEED8
:101250000000000000000000000000003006C0E0B8
:1012600000000000000000E7000000000000000097
:10127000000000E00000000000000000000000008E
:10128000000000000000001000000000000000004E
:101290000000000000000000000000070000000047
:1012A000000000000000000000000000002000001E
:1012B0000000000F0600F000000000000000000F1A
:1012C000C0000C0000000000000000000000000052
:1012D0000300000000007E3E00000000000000004F
:1012E00000000000000000000000000000000000FE
:1012F0000000000000000000000000003C3C00FF77
:10130000800000000000000FF0001C000000000042
:101310000180018000000000000000F0000F6F005D
:101320000000001BE0D80000300C000000000000AE
:1013300000000000000000000000000000000000AD
:10134000000000000198000000019FC000000000A4
:10135000000000000000000600D81C000000000093
:1013600000001FE0000000000000000000001C0062
:10137000000000000000000000000000000000006D
:10138000000000000000000000000000000000005D
:1013900000000000000000E000000000000000006D
:1013A000000000000000000000000000000003C07A
:1013B000C03C000000000000000001F800018000B7
:1013C00000000000000000000000000060000000BD
:1013D0000007FF8000000000000000000000000087
:1013E00000000000000000000000000000000000FD
:1013F000000000000000000787801FF000000000D0
:10140000000000FC000380000000000030003000FD
:101410000000000000001E0001EDE0000000037865
:101420001B0000060180000000000000000000001A
:1014300000000000000000000000000000000000AC
:10144000330000000031F000000000000000000048
:10145000000000C000078000000000000001F8004C
:1014600000000000000000000007800000000000F5
:10147000000000000000000000000000000000006C
:10148000000000000000000000000000000000005C
:1014900000003C0000000000000000000000000010
:1014A0000000000000000000000078180780000025
:1014B000000000000000000000000000000000002C
:1014C000000000000000000000000000003FC0001D
:1014D000000000000000000000000000000000000C
:1014E00000000000000000000000000000000000FC
:1014F00000000000000000000000000000000000EC
:1015000000000000000000000000000000000000DB
:10151000000000000000007FC01F0000000000006D
:101520000000000000000003E00FFC0000000000CD
:101530000000000000000001F000000000000000BA
:10154000000000000000000000000000000000009B
:10155000000000000000000000000000000000008B
:10156000000000000000000000000000000000007B
:10157000000000000000000000000000000000006B
:10158000000000000000000000000000000000005B
:10159000000000000000000000000000000000004B
:1015A00000000000000000000000F01820E0060726
:1015B0000A0C0C110F050707080C060706060C0C91
:1015C0000C0C0C0C0C0C0C0C07070C0C0C0D140F59
:1015D0000F0F0F0E0D100E050C0F0D110E100E102B
:1015E0000F0E0D0E0D150E0E0C0706070C0C070C3A
:1015F0000D0C0D0C080D0D05050C05130D0D0D0D35
:10160000080C070D0D0F0C0C0B0806080C0B0C0733
:10161000060C0B150C0C07150E0715070C07070613
:10162000060B0B070C1507150C0714070B0E060706
:101630000C0C0C0C060C070F080C0C070F0C080CFC
:101640000707070C0C060707080C1212120D0F0FE4
:101650000F0F0F0F150F0E0E0E0E050506060F0EBF
:1016600010101010100C100E0E0E0E0E0E0D0C0C95
:101670000C0C0C0C130C0C0C0C0C050506060D0DBB
:101680000D0D0D0D0D0C0D0D0D0D0D0C0D0C0000A7
:10169000000000000000000000000000000000004A
:1016A000000000000000000000000000000000003A
:1016B000000000000000000000000000000000002A
:1016C000000000000000000000000000000000001A
:1016D000000000000000000000000000000000000A
:1016E00000000000000000000000000000000000FA
:1016F00000000000000000000000000000000000EA
:1017000000000000000000000000000000000000D9
:1017100000000000000000000000000000000000C9
:1017200000000000000000007700000000007700CB
:1017300000000000000000000000000000000000A9
:101740000000000000000000000000000000000099
:101750000000000000000000000000000000000089
:101760000000000000000000000000000000000079
:1017700000070003801F007F000000000000000041
:10178000001C001C01F0000387F8000001FC01C0F0
:1017900000E001F003F800000000000038007003D2
:1017A000E000001C0000000000000000000000003D
:1017B0000000000000000000000000000000000029
:1017C0000000000000000000000000000000000019
:1017D0000000000000000000000000000000000009
:1017E00000000000000000000000000000000000F9
:1017F00000000000000000000000000000000000E9
:1018000000000000000000000000000000000000D8
:1018100000000000000000000000000000000000C8
:1018200000000000000000000000000000000000B8
:1018300000000000000000000000000000000000A8
:101840000000000000000000000000000000000098
:101850000000000000000000000000000000000088
:101860000000000000000000000000000000000078
:10187000003E00000000003E0000000000000000EC
:1018800000000000000000000000000000003180A7
:101890000000000000000000000000000000000048
:1018A000000000FFF0000000000000000000000049
:1018B00000000000000000000000038007001F007F
:1018C0007F00C6007800000000000E003801F00C18
:1018D00061CEFA300001FC00E001C001F003F80322
:1018E00018000000001C00E003E018C038000000F1
:1018F00000000000000000000000000000000000E8
:1019000000000000000000000000000000000000D7
:1019100000000000000000000000000000000000C7
:1019200000000000000000000000000000000000B7
:1019300000000000000000000000000000000000A7
:101940000000000000000000000000000000000097
:101950000000000000000000000000000000000087
:101960000000000000000000000000000000000077
:101970000000000000000000000000000000000067
:101980000000000000000000000000000000000057
:101990000000000000000000000000000000000047
:1019A0000000000000000000000000000000000037
:1019B000000000000000000000003E0000000000E9
:1019C0003E000000000000000000000000000000D9
:1019D0000000000000000031800000000000000056
:1019E000000000000000000000000000FFF0000008
:1019F00000000000000000000000000000000000E7
:101A0000000000038007003B805F00C600780000F4
:101A10000000000E003803B80C61CEDE3000017CFF
:101A200000E001C003B802F80318000000001C0029
:101A3000E0077018C038000000000000000000003F
:101A40000003C000000000000000000000000000D3
:101A50000000000000000000000000000000000086
:101A60000000000000000000000000000000C000B6
:101A70000000000000000000000000000000000066
:101A80000000000000000000000000000000000056
:101A90000000000000000000000000000000000046
:101AA0000000000000000000000000000000000036
:101AB0000000000000000000000000000000000026
:101AC0000000000000000000000000000000000016
:101AD0000000000000000000000000000000000006
:101AE00000000000000000000000000000000000F6
:101AF00000000000000000000000000000000000E6
:101B000000000000000000000000000000000000D5
:101B1000000000000000000000770000000003B893
:101B200000000000000000000000000000000000B5
:101B300000000000000000000000000000000000A5
:101B40000000000000000000000000000000000095
:101B5000000000000000780000000000000000000D
:101B60000000000000000000000000000000000075
:101B70000000000000002000000000000000000045
:101B80000000003801C03E07F00003C00000000064
:101B90007003807C00070FF000001FC03800E01FBA
:101BA00001FC00000000001C003807C00000E0003D
:101BB000000000E39C18C7F078700FC0E1CE06006B
:101BC0000000000E3F00703F07F00707F83F8FFC52
:101BD0007F83F00000000000000FE00FF801F01F0D
:101BE000F80FE07FC0FFE3FF03F8381CE01C383E2D
:101BF0007007E3F3C1C1FE07FE07F81FF80FE1FF0E
:101C0000CE07783FC3E1FE07F01EFFE7F8F81E009D
:101C100001C0001C0000000E0001F0003801CE7071
:101C200007000000000000000000000000000000AD
:101C3000000000000000001E6780000000FEFC00A5
:101C40001F800000000380383E78E0007F000FDF37
:101C5000FDF9FFFF7E19C318E700000000003F9F59
:101C6000BCF03E00000007E1F1C0780000307E00CB
:101C700003C78C1F8C61FC3F8000000007F000034D
:101C8000E0707C7C70003FF000061F0000C07030E8
:101C9000383E07000007C00F801F003E007C00F8A0
:101CA00001FFFC1FC0FFE3FF8FFE3FF9CE71C3FEB3
:101CB0000F0707F807F807F807F807F800007FFB99
:101CC00081CE07381CE07701E7001FC01C03803E6F
:101CD00007F06303C0000000003807007C0C639D20
:101CE000F461F81FC01C01C01F01FC0C6000000063
:101CF0000E007007C06301C0E0031800E39C39CFF9
:101D0000F8FC701FE0E1CE06000000000E7F80F0BE
:101D1000FF8FF80F07F87FCFFCFFC7F80000000027
:101D200000001FF01FFE01F01FFC1FF87FF0FFE313
:101D3000FF0FFE381CE01C387C7007E3F3C1C3FFC3
:101D400007FF0FFC1FFC1FF1FFCE07783FC3E1EF39
:101D50000F783CFFE7F8F81E0000E0001C000000D0
:101D60000E0003F0003801CE7007000000000000F4
:101D70000000000000010000000000000000000062
:101D80003E67C0000001FEFC001F800000000380D1
:101D9000383EFCE000FF801FFFFDF9FFFF7E39C7E2
:101DA00038E700000000003F9FBCF03E0000000745
:101DB000E1F1E0F0000030FF8003C78C3FCC67FF0B
:101DC0003F800000001FFC0007F070FCFCE0007F7B
:101DD000F0001E3F8003C0E0F0387E0E000007C018
:101DE0000F801F003E007C00F801FFFC3FF0FFE386
:101DF000FF8FFE3FF9CE71C3FF0F070FFC0FFC0FE3
:101E0000FC0FFC0FFC0000FFF381CE07381CE077CD
:101E100083C7003FE01C03807705F06303C0000028
:101E20000000380700EE0C639DBC60F017C01C0179
:101E3000C03B817C0C600000000E00700EE063016E
:101E4000C0E0031800E39C39CFFCFC701FE0E3CF37
:101E50003FC1C000000EF3C1F0F3CF781F0780FB35
:101E6000C03CF3CF7C0000030003003EF83E3F037C
:101E7000F81FFC3FFC7FF0FFE3FF1FFF381CE01C56
:101E800038F87007E3F3E1C7FF87FF1FFE1FFC3F31
:101E9000F9FFCE07783FC3E1E79E3C78FFE7F8F80B
:101EA0003F0000E0001C0000000E0003C0003800EE
:101EB00000700700000000000000000000000700A4
:101EC0000000000000000000003E67C0003FE3FE8D
:101ED000EC003C0000000003803877FCE001FFC00C
:101EE0001FFFFDD9FFFB7621C420E70000000000A2
:101EF0002F863CF000000000076000F1E000003198
:101F0000E78001EF0C3FC00F8F83800000003E3E52
:101F100000077070ECFCE0007E60001E3B8003C197
:101F2000C0F0707E0E00000FE01FC03F807F00FEFB
:101F300001FC03DFFC7FF8FFE3FF8FFE3FF9CE716A
:101F4000C3FF8F871FFE1FFE1FFE1FFE1FFE000127
:101F5000FFE381CE07381CE073C787003DE0000037
:101F60000000000000000000000000000000000071
:101F700000000003F800000000000000000000382E
:101F800000000000000000000000E0000000E39CF2
:101F900039CEDCCCE01CE0E3873FC1C000000CF38D
:101FA000C7F0E1CE381F0780F18038E1CF3C000058
:101FB0000F0003C03C78780703F81C3C7E7C71F866
:101FC000E003801F1F381CE01C39F07007E3F3E1C9
:101FD000CFCFC70F3F3F1C3C3CF81C0E073C7BC7D4
:101FE000F1E79E3C7801E738383F000000001C0014
:101FF00000000E00038000380000700700000000A1
:1020000000000000000000070000000000000000C9
:1020100000003C63C0003067E6EC003C00000000BC
:102020000383FF80CDC001E7C03E7C01D803FB766F
:1020300038473821000000000000063FF000000093
:1020400000076000F1E0000021E78C61EF0C3DC06B
:102050000E039F80000000380E000630701C3C000C
:10206000007E60001E318003C1C0F0E01E1C000035
:102070000FE01FC03F807F00FE01FC03DC00FCF886
:10208000E003800E003801CE71C387CF873F3F3F0A
:102090003F3F3F3F3F3F3F1873F3F381CE07381C6C
:1020A000E073C787FE38E000000000000000000079
:1020B00000000000000000000000000003380000E5
:1020C00000000000000000003800080000000000D0
:1020D000000000E0000000E39DFFEEC0CCE01FE048
:1020E000E787BFC1C000001CF3C7F001C0383F0F35
:1020F00000E00078E1CE1C70E07F3FF3F80038E7A5
:10210000FB83B81C1C783C7078E003803C0F381CC3
:10211000E01C3BE07007F7F3F1CF03C7073C0F1C4F
:102120001C38781C0E073C79E7F1C3FC1EF003C78E
:102130001C387F800000FF1DF03F03EE1F8FE1F78A
:102140003BF1CE71E73BEFC77E0FE1DF03FE7F3F40
:10215000CFCE0EF07F1C7F0FE0E7FC3861C000306F
:102160006780EC00FF000000003FFBFF80CDC00156
:10217000C3C3BC3C01D807BB7639C738E7000000B1
:102180000000000637B0FF1C0FEFC767FC7BC007DD
:1021900007F1C01FF0EE0C3E001CF1FF8739FF80F5
:1021A00073E7000777FF381C03877E60000631B9AC
:1021B000C0C38030E00E3800E00EE01DC03B8077E9
:1021C00000EE01DC079C00F078E003800E0038018F
:1021D000CE71C383CFC73C0F3C0F3C0F3C0F3C0F6D
:1021E0003CF3C3F381CE07381CE071EF07FF39E001
:1021F000FF0FF0FF0FF0FF0FF0FFFC0FC0FC0FC050
:10220000FC0FC39CE383FC77E0FE07F03F81FC0FEB
:10221000E03807FCE0E7073839C1DC1CEF8E0E0020
:10222000E001FFEFC0FDC01FC007879F81C0000015
:102230001CE1C77003C0F87F0FF0FF00F0F3CE1C65
:1022400070E1FF3FF3FE0078EFFB87BC1C3C780099
:102250007078E003803C00381CE01C3BC07007F73E
:10226000F3F9CF03C70F3C0F1C3C3E001C0E073C8C
:1022700079E773C1F80FE007871C3873800001FF0E
:102280009FF87F87FE3FCFE3FF3FF9CE73C73FFF45
:10229000E7FF1FF1FF87FE7F7FEFCE0E78F73E77D7
:1022A0009EF1E7FC3861C000306FFCEC00FF0000DD
:1022B00000003FFBFF80FF8001F003BC3FF9D80F17
:1022C0003B76398738C61E00000000000637B1FF94
:1022D0009C1FFFE767FC3F80070FF9E03FF8FE0C0B
:1022E0003F001DF9FB8739FF8073670007F7FF7018
:1022F000FC03877E6000063BB9C0C78031C07E38D2
:1023000000E01EF03DE07BC0F781EF03DE079FF8A1
:10231000F000E003800E003801CE71C383CFE73CAC
:102320000F3C0F3C0F3C0F3C0F3FF3C7F381CE0730
:10233000381CE070FE07FF39E1FF9FF9FF9FF9FFAE
:102340009FF9FFFE1FE1FE1FE1FE1FE39CE387FEF6
:102350007FF1FF0FF87FC3FE1FF0000FF8E0E707E3
:102360003839C1DE3CFFCF1E00E000738FF0FDC0A6
:102370000F8007879F9FFC00001CE1C67007C1F01B
:10238000770FF8FF80E07F8F3C70E3F83FF07F002D
:10239000F9DFFB87BC1FFC70007038FFC3FE3800FC
:1023A0003FFCE01C3FC07007F7F3B9CE01C7FF3810
:1023B000071FFC3FE01C0E071C71EF7BC1F80FE00C
:1023C0000F071C38F3C00001C79F7CFBCFBE79E329
:1023D00087DF3E79CE77873EFDE7CF3EF9F7CFBE68
:1023E0007979E70E0E78F7BEF3FCF1E03C3861C76F
:1023F000F3306FFCEC003C000000003FF83800FFB9
:102400008001FF07381FF9D81E3B76000000003F0F
:1024100000000000000637B1E78E3EFCF7603C3F4D
:1024200080071FFDE03EF8FE0C7FC01980FF8E7113
:10243000FF8063630003E7FFFCFC03877E63800685
:102440003F9CE0C70031C07E7000E01EF03DE07BA5
:10245000C0F781EF03DE071FF8E000FFC3FF0FFCAA
:102460003FF1CE71CFF1CEE738073807380738078C
:1024700038071FE38F7381CE07381CE070FE070F0B
:1024800039C1C79C79C79C79C79C79C7CF3EF3CF28
:102490003CF3CF3CF39CE38FBE7CF3EF9F7CFBE7E8
:1024A000DF3EFBFF9F7CE0E7073839C1DE3CFBEFF6
:1024B0001E00E0007387FC7B803F800703999FFC30
:1024C000000018E1C0700F81F8E70F7CF3C1E07FD6
:1024D0008F3C0003C000000F01F1DFF18F1E1FFCD5
:1024E00070007038FFC3FE387F3FFCE01C3FE07097
:1024F00007F7F3BDCE01C7FE38071FF81FF01C0E0B
:10250000071EF1EF7BC0F007C01E070C38F3C000B8
:10251000003F9E3CF3CF1E70E3878F3C39CE7F0790
:102520003C78E78F3C79E3CF1E7878070E0E38E3CE
:10253000BEE1F871C0787861E7FF306700EC0038E1
:1025400000000000038038007B8000FF8F381FF9F7
:10255000D83C3B76000000003F000000000006333E
:1025600031E00F3C7C7760781F00001EFFFC1C717F
:10257000FF0C7FE01980FF9EF0038063E300000002
:1025800070FC7803873E6380061F1EF0CE1C339FCD
:102590003CE1C0003C7878F0F1E1E3C3C7878F0FDE
:1025A0001FF8E000FFC3FF0FFC3FF1CE71CFF1CE6B
:1025B000F7380738073807380738070FC39E738185
:1025C000CE07381CE0707C070739E03F83F83F8373
:1025D000F83F83F803C73CF38738738738739CE36D
:1025E0008F1E78F3C79E3CF1E78F3C7BFF9E7CE01B
:1025F000E7073839C1CE38F1E71C00E0007381FCF1
:1026000003BC7FFC0703801FFC07E038E1C0700FAC
:10261000817CC7003CF3C1E0F3C7FC0003F8000075
:102620007F03C1DEF18F1E1FFE70007038FFC3FEF6
:10263000387F3FFCE01C3FE07007FFF39DCE01C7F1
:10264000FC38071FF007F81C0E071EF0EE3B81F860
:1026500007C03C070E3800000000FF9C1CE00E0E77
:102660007FE387073839CE7F073870E7073839C1ED
:10267000CE0E707F070E0E3DE3BEE1F87BC0F07812
:1026800061E7FF306FF8EC0078000000000380384D
:10269000000778F03FCE381C01D8783B7600000068
:1026A000003F0000000000000001FC07383FF76019
:1026B000F01F00071CC3FC1831FF0C73E01980C029
:1026C0001CE0039FE3E30000007000000387066343
:1026D0008000000E700E3C073F00E3C0E03C7878BD
:1026E000F0F1E1E3C3C7878F0FFC00E000FFC3FFF9
:1026F0000FFC3FF1CE71C381CE773807380738071A
:10270000380738070FC3BC7381CE07381CE0707CD4
:10271000070F39F0FF8FF8FF8FF8FF8FF83FFF3872
:1027200003FF3FF3FF3FF39CE38E0E7073839C1C0B
:10273000E0E707383BFF9CFCE0E7073839C1CF787A
:10274000E0E7BC00E001FFE0FC077E7BFC070380C4
:1027500001C007E038E1C0701F003DC7001CE1C3A5
:10276000C0F3C3FC0001FF3FF3FE03C19CF38FFEE7
:102770001C1E78007078E003803C7F381CEE1C3C07
:10278000F07007FFF39FCF03C7003CEF1CF000F889
:102790001C0E070FE0FE3F81F8038078070E38001B
:1027A000000001FF9C1CE00E0E7FE387073839CE46
:1027B0007F873870E7073839C1CE0E703FC70E0EDD
:1027C0003DE3FFE0F07BC1F0F060F67F306FF8ECA6
:1027D0000078000000000380380007FDF807CE3CB9
:1027E0003C01D8F03B76000000003F7FFFFFFFC0B8
:1027F000000000FF07383FF761F00E00071C80E083
:102800001C70380079E01DF9C01CE0039FF37700CD
:102810000000700000038706600000000E701C6C52
:10282000073B01C6C1E03FF87FF0FFE1FFC3FF8730
:10283000FF1FFC00F000E003800E003801CE71C3E2
:1028400083CE7F3C0F3C0F3C0F3C0F3C0F1FE3F847
:10285000F381CE07381CE0703807FF38F9FF9FF985
:10286000FF9FF9FF9FF8FFFF3803FF3FF3FF3FF3A0
:102870009CE38E0E7073839C1CE0E7073838001DC4
:10288000DCE0E7073839C1CF78E0E7BC00E001FFC2
:10289000E0DC077E71FC07038001C007E038F3C06D
:1028A000703E001DFFC01CE1C3C0E1C01C00007FE2
:1028B0003FF3F803819DF39FFF1C0E783C7078E096
:1028C00003803C07381CEF1C38F07007BEF38FCF35
:1028D00003C7003CFF1C7878381C0F0F0FE0FE3F49
:1028E00083FC0380F0070E3800000001E39C1CE02D
:1028F0000E0E700387073839CE7F873870E70738A8
:1029000039C1CE0E701FE70E0E1FC3F7E1F83F81ED
:10291000E0F060F000306780EC0078000000000319
:1029200080380006FDFBC1CF3C3C01D9E03B76007E
:102930000000001E7FFFFFFFC00000007F8F3838BF
:102940000761E00E00071F81E03EF9FF007CE01CFC
:10295000F1C01EF0039FF3770000007000000387B2
:1029600006600000001EF038CC0E07038CC3E07F29
:10297000FCFFF9FFF3FFE7FFCFFF9FFC00F078E0DB
:1029800003800E003801CE71C383CE3F3C0F3C0F55
:102990003C0F3C0F3C0F3FF3F0F3C3CF0F3C3CF038
:1029A000F03807FE3879E39E39E39E39E39E39FF1C
:1029B0008038038038038038039CE38E0E70738365
:1029C0009C1CE0E7073838381F9CE0E7073839C11E
:1029D000C7F0E0E3F8000000E70EDC076671F807D7
:1029E000038001C0000070F3C070780F3DFFCF3C42
:1029F000F3C3C0F3CE3C00000F3FF3C000019FF7CC
:102A00001FFF1C1E7E7C70F8E003801F1F381CEF28
:102A10003C38787007BEF387CFCFC7003FFF1C3C20
:102A20007CF81C0F9F0FE0FE1F879E0381E00706C6
:102A30003800000001C79E3CF3CF1E79E3878F3832
:102A400039CE73C73870E7073C79E3CF1E7001E7D2
:102A50000F1E1FC1F7C3F83F83C07861E0003067E5
:102A6000E6EC007800000000038038000ECD9BE704
:102A7000C73E7C01DBC03B76000000000000000088
:102A80000000000000078E3C7CF763C00E00071FAB
:102A9000BDE03FF9FF007FE00E03800E7003803839
:102AA0000E00000000000003CF06600000001CE0E4
:102AB00038FE0E0E038FE7C07FFCFFF9FFF3FFE740
:102AC000FFCFFFBC1C00FCF8E003800E003801CEF5
:102AD00071C387CE1F3F3F3F3F3F3F3F3F3F3F3C9C
:102AE000F3F3F3E7CF9F3E7CF9F03807FC3839C7A2
:102AF0009C79C79C79C79C79C3CF3CF3CF3CF3CF7B
:102B00003CF39CE38F1E7073C79E3CF1E78F3C78CB
:102B1000381F3CF1E78F3C79E3C7F0F1E3F800E0C0
:102B200000E70FFC0E6679FC07878001C1C00E70BC
:102B3000F3C070F00F3C070F7CFBC3C0F3CF7C7079
:102B4000E0030003000381DFEF1C071FFE3FFC7F53
:102B5000F0FFE3801FFF381CEFFC383C7FE73E733B
:102B600087C7FF87001FFE1C3C7FF81C0FFF07C0B4
:102B70007C1F079E0381FFE7073800000001EF9FDD
:102B80007CFBCFBE7DE387DF3839CE71E73870E755
:102B9000073EF9F7CFBE7079E70F3E0F81F7C3FC10
:102BA0001F07807861E0003063FEECE07839C3876E
:102BB0000E038038000ECD9BFFC39FFFFDDBFFFBA4
:102BC0007600000000000000000000000001E79C0B
:102BD0003EFEF767800E00071FFFFF9FF0380C3F97
:102BE000C00F8F80073800003E3E000007FF000046
:102BF00003DF066000000039C070FE1C1C070FEFE9
:102C000080701CE039C07380E701CE03BC1FFC7FDD
:102C1000F8FFE3FF8FFE3FF9CE71C3FF8E1F1FFE4B
:102C20001FFE1FFE1FFE1FFE3871FFE3FFCFFF3F99
:102C3000FCFFF03807003BF9EF9EF9EF9EF9EF9E9D
:102C4000F9EFEF3EF3EF3EF3EF3EF39CE38FBE7000
:102C500073EF9F7CFBE7DF3EF8381F7CF3E79F3C78
:102C6000F9E7C3E0FBE1F000E000E70FF80E7E3F7C
:102C7000FE0787800001C00E707F8070FFC7F807D5
:102C800007F87F83807F8FF870E0000000000381E9
:102C9000DFFE3C079FFE1FF87FF0FFE3800FFE384A
:102CA0001CE7F8383C7FE73E7383C3FF07000FFF44
:102CB0009C1E3FF01C07FE07C07C1F0F0F0381FF07
:102CC000E7073800000001FFDFF87F87FE3FC3837E
:102CD000FF3839CE71E73870E7071FF1FF87FE70C4
:102CE0007FE7CFFE0F81F7C79E1F07FC3861C0004A
:102CF0003061FEECE07039C3870E0383FF801CFD5A
:102D0000F9FF839FFFFDDBFFFB7600000000000062
:102D100000000000000001FF9C1FFFE767FC0E00A1
:102D2000070FFBFF8C60380C0FC007FF000738004F
:102D3000001FFC000007FF000003FF06600000000A
:102D400039C0E00C383F0F00CF00F01FE03FC07FDC
:102D500080FF01FE03F81FFC3FF0FFE3FF8FFE3F03
:102D6000F9CE71C3FF8E0F0FFC0FFC0FFC0FFC0F91
:102D7000FC0003FFC1FF87FE1FF87FE03807003B20
:102D8000F9FFDFFDFFDFFDFFDFFDFFFE1FE1FE1F9F
:102D9000E1FE1FE39CE387FC7071FF0FF87FC3FE29
:102DA0001FF0000FF8FFE7FF3FF9FFC3E0FFC1F09E
:102DB00000E000E707F81C7E1FDC0787800001C0E9
:102DC0000E703F0070FFC3F00703F03F03803F0722
:102DD000F070E0000000000381CEF83C079FFC0F7C
:102DE000E07FC0FFE38003FC381CE3F0381E7FE780
:102DF0003E7383C1FE070007FF9C1E1FE01C03FCFF
:102E000007C07C1F1E078381FFE707380000000012
:102E1000FFDDF03F03EE1F8381F73839CE70F738BE
:102E200070E7070FE1DF03EE703FC7C7EE0700E36F
:102E30008F0F1F07FC3861C0003FE0FEFCE0F03957
:102E4000C3870E0383FF801CFDF8FF000FFFFDFB0F
:102E5000FFFF7E00000000000000000000000000F6
:102E6000FF000FEFC7E7FC0E000707F3BF80003835
:102E70000C07C001FC000000000007F0000007FF85
:102E8000000003FF06600000000000E00C383F0E69
:102E900000CE00F01FE03FC07F80FF01FE03F81F5F
:102EA000FC1FC0FFE3FF8FFE3FF9CE71C3FE0E0F84
:102EB00007F807F807F807F807F80007FF80FF038F
:102EC000FC0FF03FC038070039F0FFCFFCFFCFFC0C
:102ED000FFCFFCFEFC0FC0FC0FC0FC0FC39CE383C4
:102EE000F87070FE07F03F81FC0FE0001FF07EE3FA
:102EF000F71FB8FDC3E0EF81F00000000000C01C28
:102F00003C000003870000004000000000000000BB
:102F10000000000000000000000000200000000091
:102F20000000E003C00000000000000000000000FE
:102F30000000000000000000000000000000000091
:102F400000038000000000000000000000000000FE
:102F50000000070038000000000000000000000032
:102F600000000700000E0000000000000001C0008B
:102F70000E000000000000000000001E00003C6386
:102F8000C0000000000020F0084000000383FF8024
:102F90001C78F000000000000000000000000000AD
:102FA0000000000000000000000000000000000021
:102FB0000000070200000000000C39C00000000003
:102FC0000000000000000000000000038006600F09
:102FD000800000000000000000000F1E0000000044
:102FE000000000000000000000000F800000000052
:102FF00000000000000000000000000000000000D1
:1030000000000000010000000000000000000000BF
:10301000000000000000000000000000000007C0E9
:1030200000000000000000000000000000000000A0
:103030000000000000080000000000000003C0E0E5
:1030400001E00000000000C00000000003C7000015
:1030500001C00000000000000000000000000000AF
:1030600000000000E0000000000000F007C00000C9
:103070000000000000000000000000000000000050
:103080000000000000000000000000000000000040
:10309000000000000000000000000007C0F8000071
:1030A00000000000000000000000079F00001E005C
:1030B00000000000000001C0000E00000000000041
:1030C000000000001E00003E67C00000000000E09D
:1030D000F039C0000003803800000000000000004C
:1030E00000000000000000000000000000000000E0
:1030F00000000000000000000000000706000000C3
:1031000000000C3FC00000000000000000000000B4
:1031100000000000038006600B800000000000003B
:103120000000000FBE0000000000000000000000D2
:103130000000000B80000000000000000000000004
:10314000000000000000000000000000000000007F
:10315000000000000000000000000000000000006F
:103160000000000000000005C0000000000000009A
:10317000000000000000000000000000000000004F
:1031800000000000000003C0E001E00000000000BB
:10319000000000000001CE000001800000000000DF
:1031A00000000000000000000000000000C000005F
:1031B000000000007E3F80000000000000000000D2
:1031C00000000000000000000000000000000000FF
:1031D00000000000000000000000000000000000EF
:1031E0000000000007C0F8001FFE00000000000003
:1031F00000000007FF00001E0000000000000001AA
:10320000C0000E000000000000000000007C000074
:103210003E67C00000000000C7F03180000003805E
:103220003800000000000000000000000000000066
:10323000000000000000000000000000000000008E
:1032400000000000070600000000000C3FC0000066
:1032500000000000000000000000000000038006E5
:1032600060038000000000000000000007FC000078
:1032700000000000000000000000000003800000CB
:10328000000000000000000000000000000000003E
:10329000000000000000000000000000000000002E
:1032A000000000000000000000000000000000001E
:1032B00001C000000000000000000000000000004D
:1032C0000000000000000000000000000000000FEF
:1032D00080E007C00000000000000000000001CEF8
:1032E00000000000000000000000000000000000DE
:1032F000000000000000000000000000003FFF0090
:1033000000000000000000000000000000000000BD
:1033100000000000000000000000000000000000AD
:103320000000000000000000000000000007C0F8DE
:10333000001FFE00000000000000000003FC000071
:103340001C0000000000000001C0000E0000000092
:103350000000000000007C00001E678000000000EC
:103360000007E000000000038038000000000000BB
:10337000000000000000000000000000000000004D
:103380000000000000000000000000000007060030
:10339000000000000C1F8000000000000000000082
:1033A000000000000000038006601F800000000095
:1033B000000000000003F800000000000000000012
:1033C00000000000001F800000000000000000005E
:1033D00000000000000000000000000000000000ED
:1033E00000000000000000000000000000000000DD
:1033F0000000000000000000000FC00000000000FE
:1034000000000000000000000000000000000000BC
:1034100000000000000000000F80E007C000000076
:10342000000000000000000000000000000000009C
:10343000000000000000000000000000000000008C
:103440000000000000000FFC000000000000000071
:10345000000000000000000000000000000000006C
:10346000000000000000000000000000000000005C
:10347000000000000000000000000000000000004C
:10348000000000000000000000000000000000003C
:10349000000000000000000000000000000000002C
:1034A00000000060000000000000000000000000BC
:1034B000000000000000000000000000000000000C
:1034C00000000000000000000000000000000000FC
:1034D000000000000000000000000000000C0000E0
:1034E00000000000000000000000000000000000DC
:1034F00000000000000000000000000000000000CC
:1035000000000000000000000000000000000000BB
:1035100000000000000000000000000000000000AB
:10352000000000000000000000000000000000009B
:10353000000000000000000000000000000000008B
:10354000000000000000000000000000000000007B
:10355000000000000000000000000000000000006B
:1035600000000000000031C397206D697474696722
:1035700020616E74697070656E21004269747465B3
:1035800020616C6C652076696572204B7265697389
:1035900065006B616C696272696572656E00546F7B
:1035A00075636873637265656E0053656B2E004DBD
:1035B000696E2E005374642E00546167004D6F6E67
:1035C0002E004A61687200446174756D2F556872EF
:1035D0007A656974207374656C6C656E002564008F
:1035E000536F004D6F004469004D6900446F004601
:1035F00072005361000025640025530062726175FA
:103600006E00626C617500677261750067656C625F
:1036100000255320323025303264004D6F6E6174C6
:10362000736B616C656E64657200005550AAA0A54D
:1036300090FFF0F5D0FAE0E5E400273011241FBE3A
:10364000CFEFD8E0DEBFCDBF13E0A0E0B1E0ECE506
:10365000FAE702C005900D92A034B107D9F714E043
:10366000A0E4B3E001C01D92A53EB107E1F716E367
:10367000CCE3D6E304C02297FE010E94283DCA3362
:10368000D107C9F7F9D40C9480390C940000FC01DF
:103690008F3F910509F048F48031910518F084E0DE
:1036A00090E00CC080E090E009C080E1E030F807D5
:1036B00018F08CE090E002C088E090E020E130E07B
:1036C000281B390B02C0F695E7958A95E2F7E05C76
:1036D000FE4F8081281B3109C9010895EE27FF277D
:1036E000E81BF90BE823F923EF3FF10509F048F453
:1036F000E031F10518F024E030E00CC020E030E0CB
:1037000009C080E1E030F80718F02CE030E002C09A
:1037100028E030E0022E02C0F695E7950A94E2F721
:10372000E05CFE4F808121503040280F311DC901DF
:103730000895292FA0E4B2E0FD01E80FF11D80817A
:1037400030E0A20FB31F2C9130E0280F311DC901CA
:1037500008959C01409142035091430380914A0394
:1037600090914B03481B590B460F571F80E493E081
:10377000B9010C9418250F931F93CF93DF93EC019D
:10378000109249031092480310924B0310924A037F
:103790008091640380FD28C000E411E020EF30E058
:1037A000235030400350104080E493E062E070E02A
:1037B00043E150E05BD7D0936A03C09369038091E3
:1037C00065038D7F8093650380E493E0BE010E94D2
:1037D000CC29C095D095D0936803C0936703DF913F
:1037E000CF911F910F91089500EF10E020E431E098
:1037F000D7CFCF92DF92EF92FF920F931F937C016E
:1038000069010E941825C701B601A8010E94FA2784
:103810001F910F91FF90EF90DF90CF900895CF927E
:10382000DF92EF92FF920F931F937C0169010E9438
:103830001825F70185A1806185A3C701B601A801FC
:103840000E944125C7010E946125C70102960E947E
:103850006125C7010E9479261F910F91FF90EF907B
:10386000DF90CF9008958F929F92AF92BF92CF92A8
:10387000DF92EF92FF920F931F934C015B0197E64B
:10388000C92E93E0D92E84E195EA90936803809342
:10389000670390936A0380936903F60132978081EE
:1038A0008D7F808389ED9FEFC80ED91EC60160E031
:1038B00070E040E050E020EF30E08401B0DF80E4D1
:1038C000E82E81E0F82EA7014A195B09C60160E0E5
:1038D00070E020EF30E08501A2DFE818F908EA186F
:1038E000FB08C60160E070E0A40122E030E087013F
:1038F00096DFC6016EEE70E0A40122E030E08FDFBB
:103900001092680310926703C6016DE872E00E948E
:10391000312C82E0809366031F910F91FF90EF900E
:10392000DF90CF90BF90AF909F908F900895AF920F
:10393000BF92CF92DF92EF92FF920F931F93CF939C
:10394000DF9383E190E062E070E08DDF80E493E05C
:1039500068E770E040E050E00E94182580E493E0C2
:103960006EEC70E00E94052C8FEF9FEF04DF109249
:1039700049031092480310924B0310924A0380E0CF
:1039800090E0F9DEFEEDAF2EF0E0BF2E6501CAEA51
:10399000D0E0F6018591949190936803809367033A
:1039A00040E451E04C1B5D0B0CE711E00C1B1D0BC0
:1039B00080E493E0BE01EC969E01E6E0EE2EF12C51
:1039C0000E94982882E090E0C80ED91EC055D040D1
:1039D00098EEC91690E0D906E1F6C8E2D0E0F5010C
:1039E00085919491909368038093670380E493E0BA
:1039F000BE01EC96AE012EE130E00E94422982E049
:103A000090E0A80EB91EA89798EEA91690E0B90606
:103A100031F780E098EF9093680380936703E0901C
:103A20005E03F0905F0380915A0390915B03E81A64
:103A3000F90AC0E0D0E015C06091580370915903B5
:103A400040915A0350915B034C0F5D1F9E01260F5E
:103A5000371F00915E0310915F0380E493E0C9DE9D
:103A60002A96CE15DF0544F3E70115C000915A03ED
:103A700010915B0360915C0370915D03AE01400F98
:103A8000511F20915803309159032C0F3D1F80E4A2
:103A900093E0AFDE2A971C161D0644F38FEF97E0E4
:103AA0009093680380936703E70115C000915A0360
:103AB00010915B036091580370915903AE01400F60
:103AC000511F20915C0330915D032C1B3D0B80E462
:103AD00093E08FDE2A971C161D0644F3C0E0D0E069
:103AE00015C060915C0370915D0340915A03509141
:103AF0005B034C0F5D1F9B012C1B3D0B00915E0374
:103B000010915F0380E493E074DE2A96CE15DF0502
:103B100044F3DF91CF911F910F91FF90EF90DF90D1
:103B2000CF90BF90AF900895809113018F5F8093E5
:103B300013018C33C1F410921301809114018F5F33
:103B4000809314018C3379F4109214018091150143
:103B50008F5F80931501883131F41092150186E151
:103B600091E00C94AF2F08951F920F920FB60F9211
:103B700011242F933F934F935F936F937F938F9372
:103B80009F93AF93BF93EF93FF93CEDFFF91EF919E
:103B9000BF91AF919F918F917F916F915F914F9165
:103BA0003F912F910F900FBE0F901F901895EF929D
:103BB000FF920F931F93DF93CF93CDB7DEB7649738
:103BC000DEBFCDBF8DB79EB70A979EBF8DBFEDB745
:103BD000FEB731967E010894E11CF11CADB7BEB76B
:103BE0001296FC92EE92119788EE90E09383828376
:103BF00080911501992787FD909595838483809105
:103C00001401992787FD90959783868380911301EE
:103C1000992787FD9095918780870E948B398DB772
:103C20009EB70A969EBF8DBF00E413E0C80168E707
:103C300070E042E251E0FCD6C801B7010E94B52B0A
:103C40006496DEBFCDBFCF91DF911F910F91FF90A2
:103C5000EF900895EF92FF920F931F93CF93DF930E
:103C6000EC014881598141155105E9F08C819D8114
:103C700090936803809367034B5050400A811B81E7
:103C8000055F1F4F80E493E065E070E02BEE30E0CD
:103C9000AAE0EA2EF12C0E9471278C819D818095EB
:103CA00090959D838C83DF91CF911F910F91FF9011
:103CB000EF9008950F931F93CF93DF938C01EB0147
:103CC000209741F0C8010E9482390196080F191F00
:103CD0002197F6CFC801DF91CF911F910F910895E1
:103CE000EF92FF920F931F93DF93CF93CDB7DEB781
:103CF0006497DEBFCDBF09E613E010926A0310920D
:103D00006903F801349780818D7F80838FEF9FEF67
:103D1000909368038093670386E191E00E94462FA9
:103D2000682F772767FD709589EF90E0C3DF00D09B
:103D300000D000D0EDB7FEB731967E010894E11CAB
:103D4000F11CADB7BEB71296FC92EE92119727E424
:103D500031E033832283958384830E948B392DB78E
:103D60003EB72A5F3F4F3EBF2DBF09521040C801EA
:103D700068E770E040EF50E05BD6C801B7010E94F1
:103D8000B52B60911701772767FD709561507040E2
:103D90008AE790E08FDFADB7BEB71C97BEBFADBF5F
:103DA000EDB7FEB731961296FC92EE92119727E38B
:103DB00031E03383228320911601332727FD30958C
:103DC000358324839783868380911901992787FD02
:103DD00090959187808780911801992787FD90950C
:103DE000938782870E948B392DB73EB7245F3F4F60
:103DF0003EBF2DBFC80168E770E049E051E018D62A
:103E0000C801B7010E94B52B6496DEBFCDBFCF912C
:103E1000DF911F910F91FF90EF9008952F923F92A5
:103E20004F925F926F927F928F929F92AF92BF92CA
:103E3000CF92DF92EF92FF920F931F93DF93CF9376
:103E400000D000D0CDB7DEB7882E809116019091BA
:103E50001701A0911801B091190189839A83AB834E
:103E6000BC8310E005C0CE0101960E94AF2F1F5FFA
:103E70001815CCF310E0992401E0CE010196612FD2
:103E80000E9476348111902A1F5F143011F0000FC8
:103E9000F4CF992011F410E005C0892D90E01EDCCC
:103EA000182F1F5F292C3324C10143DC082F8823DE
:103EB00009F401E0812F992787FD9095880F991FBC
:103EC000FC01E859FF4F45905490FC01E45BFE4F24
:103ED000659074905092680340926703C0904203CB
:103EE000D090430380914A0390914B03C81AD90A9A
:103EF00082E290E0C80ED91E84E10802500111242C
:103F0000AC0CBD1C8EED9FEFC80ED91E91E089163A
:103F100099F4992069F0D0927503C0927403B0921D
:103F20007703A0927603709279036092780304C0BD
:103F3000109275031092740380E493E060E170E0E6
:103F4000A60120EE30E08501E6E0EE2EF12C0E9485
:103F50009828709268036092670380E493E060E1C0
:103F600070E0A60120EE30E0B3E0EB2EF12CEBD6B2
:103F700050926A0340926903809165038D7F80931C
:103F8000650384E090E0C80ED91E80E493E06EE102
:103F900070E0A6014DD5682D772767FD70958BE9F8
:103FA00091E088DEBC0180E493E00E94052C8EE164
:103FB00090E068E170E0CDDB9920C1F110E8EE24DB
:103FC000FF24812F90E082219321892B31F112303F
:103FD00079F0133018F41130D9F405C0143069F0B9
:103FE0001830B1F40FC080E493E06FE871E00EC0C8
:103FF00080E493E063E871E009C080E493E067E760
:1040000071E004C080E493E06AE671E00E94052C50
:104010008EE190E064E170E09CDB16950894E11C71
:10402000F11C98E0E916F10461F60BC080E493E01E
:104030006EE571E00E94052C8EE190E064E170E095
:1040400088DB80E190E063E170E083DB2496DEBFF3
:10405000CDBFCF91DF911F910F91FF90EF90DF9037
:10406000CF90BF90AF909F908F907F906F905F9018
:104070004F903F902F900895EF92FF920F931F93D0
:10408000DF93CF9300D000D0CDB7DEB78AE793E0BF
:1040900060E070E040EC50E00E947A3B80E493E006
:1040A00060E027D383E793E00E945B2C10928000AE
:1040B0008DE08093810088E09DE390938900809358
:1040C000880082E080936F0081E083BF86EF809359
:1040D00064007894CE01019660EC70E044E050E01A
:1040E0000E947A3B8AE394E06CEC70E048E050E098
:1040F0000E947A3B89818831C0F58A8181508F3155
:10410000A0F58B8181508C3080F58C81843668F5E8
:1041100089819A81AB81BC818093150190931601AE
:10412000A0931701B0931801109214010BEC10E04A
:10413000B8E0FB2E13C0C8010E948A3B8095015055
:104140001040882359F090E0A2DA90E1981BFF0C10
:10415000FF0CFF0C9F0D9093140104C0FA942FEFF5
:10416000F21649F787E380931301E0901401FF24CE
:104170000E2D10E080911401992787FD9095081766
:10418000190709F43EC085E191E060EC70E044E07D
:1041900050E00E94923B40911401442399F424EC96
:1041A00030E0F999FECF32BD21BDF89484E18FBB98
:1041B00086E18FBB78942F5F3F4F80E02C3C38071F
:1041C00081F71DC0F999FECFC801A3E095958795A9
:1041D000AA95E1F78C539F4F92BD81BD0770107077
:1041E00081E090E002C0880F991F0A95E2F7809560
:1041F00080BDF89484E28FBB86E28FBB78941FBAAF
:10420000E42E409116012F2D30E0842F992787FD51
:10421000909528173907D9F0F42E89DB80E493E0D4
:104220006AEA75E10E94312C1092660380E493E003
:1042300060E170E049E150E0FBD380E0EFDD81E038
:10424000EDDD82E0EBDD82E08093660349DD83E70C
:1042500093E00E94612C8823A9F183E793E061E059
:104260000E94792C805092405CF40E94962D882305
:1042700021F18AE394E06CEC70E048E050E012C079
:1042800083E793E060E00E94792C80509240B8F47C
:104290000E944C36882349F08AE793E060E070E0A2
:1042A00040EC50E00E94923B08C08AE793E060E057
:1042B00070E040EC50E00E947A3BFF240DC00E9469
:1042C000CB32FBCF8FEF9FEF909368038093670310
:1042D0006EDC84E793E0BEDC83E793E06EEF7FEF74
:1042E0000E94AB2C45CF9BB1282F2C7F9370292B9C
:1042F0002BB995B183709C7F982B95B94198419AC1
:1043000008954298F0DF429A08951F93182F892F3D
:10431000EADF812FE8DF1F9108950F931F93CF935A
:10432000DF93EC018B0160E070E020E030E0CB0136
:10433000BA01A90198010E94533C9B01AC0161158F
:1043400071058105910509F44EC0E62FBB27A52F05
:10435000942F832F682FCA01AA27BB27782F2111FA
:104360006F5F61117F5F4D2F5527CE019070481709
:104370005907B9F49BB12C2F8C2F8C7F9370892B0C
:104380008BB985B123708C7F282B25B94198419A30
:104390004198419AE150D1F76150C1F77150B1F79E
:1043A00022C09BB1242F842F8C7F9370892B8BB9D3
:1043B00085B123708C7F282B25B94198419A9BB1F8
:1043C0002C2F8C2F8C7F9370892B8BB985B1237008
:1043D0008C7F282B25B94198419AE15011F7615003
:1043E00001F77150F1F6DF91CF911F910F91089570
:1043F000EF92FF920F931F93F62E172FE42E052FA7
:1044000080DF812F70DF8F2D6EDF802F6CDF8E2D90
:104410006ADF1F910F91FF90EF900895EF92FF9246
:104420000F931F93CF93DF93FC0116C031967F014A
:104430000894E11CF11CE4918E2F63DFE701102F3B
:1044400005C0FE012196E4918E2F4DDF1150C9F772
:104450000150F701E00FF11D0491002339F7DF91BE
:10446000CF911F910F91FF90EF900895CF93DF931D
:10447000DC01CD91DC911197FE018191282F33272A
:1044800027FD30951196FC93EE9327FF2FC025FF53
:1044900017C0322F22273295307F8981482F552728
:1044A00047FD50954F73507086E0440F551F8A9515
:1044B000E1F7422B532B31961196FC93EE9308C0F3
:1044C000A90176E0440F551F7A95E1F7407C5770BB
:1044D000ED91FC9111978191282F332727FD30957D
:1044E0002F733070242B352BED93FC93C901DF9192
:1044F000CF910895DC01ED91FC911197AF014F5FD1
:104500005F4F11965C934E93E4912E2F30E0E7FFBE
:1045100031C0E5FF19C0322F22273295307F4F5F1F
:104520005F4F11965C934E9341505040FA01849135
:10453000482F50E04F73507066E0440F551F6A9546
:10454000E1F7422B532B08C0A90126E0440F551F69
:104550002A95E1F7407C5770ED91FC9111973196C7
:10456000ED93FC933197E4912E2F30E02F73307050
:10457000242B352BC90108950F931F93962F272FB6
:10458000142F052F8AE2492F522F32DF8BE2612F41
:10459000702F412F502F2CDF8CE2B3DE1F910F9133
:1045A00008950F931F93CF93DF93EC01162F0CA167
:1045B000017067FF18C086E3A4DE9CA1892F847078
:1045C0008964990F990F990F9071892B212F30E0F1
:1045D000402F50E024273527E5E0220F331FEA95CE
:1045E000E1F7822B80DE16FF0FC06C857D85488940
:1045F00059898AE2FDDE6E857F854A895B898BE277
:10460000F7DE8CE27EDE0BC014FF09C06881798181
:104610004A815B8120E0011121E0CE01ADDFDF9115
:10462000CF911F910F910895FC0184A186FF0FC0C7
:104630002681378187FF07C082819381880F991F68
:10464000821B930B01C0C901938382830895248147
:10465000358187FF07C080819181880F991F821B58
:10466000930B01C0C9019183808308950F931F9319
:10467000CF93DF93FC01E901A5A1A4FF0EC0208523
:104680003185620F731F82859385480F591FC20FB2
:10469000D31F080F191FAF7EA5A384A180FD24C0DE
:1046A00020E431E080EF90E077FF02C060E070E04E
:1046B000718F608F57FF02C040E050E0538F428FF0
:1046C0000197C817D9070CF4CE01958F848FC901C3
:1046D0000197081719070CF4C801978F868FDF918F
:1046E000CF911F910F91089520EF30E080E491E089
:1046F000DBCFFF920F931F93CF93DF93EC016CA35B
:104700001DA21EA260E070EE40E050EE20E030E21C
:1047100000E010E2ABDF198618861B861A8688B186
:104720008F6188B987B18F6187B98AB18C6F8AB977
:1047300084B1836084B9449A80E29EE40197F1F7E2
:10474000449880E69AEEFC013197F1F7449A01977C
:10475000F1F7439884EF91E0E0E9F1E03197F1F768
:104760000197D1F781E592E059DE8EE192E056DEC5
:1047700014E0F12E00E010E089EFC3DD8F2DB3DDF2
:1047800081E092E04BDEF6940F5F1F4F033011057E
:1047900099F781E1B6DD80EB94E0E0E9F1E0319753
:1047A000F1F70197D1F786EF91E038DE439A18A62A
:1047B0001FA28FEF9FEF9AA789A78DA18D7F8DA351
:1047C000DF91CF911F910F91FF900895FC01208DF3
:1047D000318D84859585A901481B590B11A210A222
:1047E0001416150624F43587248751A340A3248D7D
:1047F000358D808991892817390714F4318B208BE6
:1048000080899189019624853585821B930B958B30
:10481000848B20E0181619060CF421E0822F0895ED
:104820004F925F926F927F928F929F92AF92BF92C0
:10483000CF92DF92EF92FF920F931F93CF93DF936C
:10484000EC017B016A018901C1DF882309F4AFC053
:10485000CE010296BBDF882309F4A9C028A139A1A3
:104860004AA15BA18CA1682F70E0DB01A870B07039
:1048700083FF03C0CA01A9019C01F901E00FF11FE8
:104880004C9DC0014D9D900D5C9D900D1124E80F35
:10489000F91F6C887D88AE88BF88AB2B19F0C501E5
:1048A00053013C018F01B3E015950795BA95E1F7E7
:1048B0000E0D1F1DA7E0EA2EF12CEE22FF2226018D
:1048C000461857084398E3E075956795EA95E1F730
:1048D0006770606FCE0165DEF80144919701209505
:1048E00030952770307081E090E002C0880F991FEA
:1048F0002A95E2F7982E842E63018DA1292D30E0B0
:10490000482D50E081FF05C024233523232B59F087
:1049100004C024233523232B19F08FA198A502C0AE
:1049200089A59AA5F2DC0894E11CF11C0894C10841
:10493000D108C114D10499F0892D90E095958795FF
:10494000982E8823D1F60F5F1F4FF801849128EF2E
:104950003FEFE20EF31E882E50E8952ECECF08943E
:10496000A108B108A114B10489F09701240D351DE7
:10497000C90143E0959587954A95E1F7080F191FFE
:1049800087E0E82EF12CE222F322A6CF888D998DC4
:104990009D878C878A8D9B8D9F878E878C8D9D8D23
:1049A000998B888B8E8D9F8D9B8B8A8B439ACE01A2
:1049B0003BDEDF91CF911F910F91FF90EF90DF9041
:1049C000CF90BF90AF909F908F907F906F905F90AF
:1049D0004F900895FC0120813181808D918D2817A1
:1049E0003907A4F0848D958D821793077CF042815E
:1049F0005381828D938D4817590744F020E0868DAE
:104A0000978D841795071CF021E001C020E0822FCC
:104A10000895CF93DF93EC01DDDF882331F0CE01E1
:104A200060E3BFDD8FA198A570DCDF91CF91089581
:104A3000FC0125A124FF0FC080819181860F971F63
:104A40009183808382819381840F951F93838283D6
:104A50002F7E25A3089580859185860F971F9183CA
:104A6000808382859385840F951F93838283089525
:104A70000F931F938C01DCDFC801CBDF1F910F91D7
:104A80000895FC0125A124FF0FC080819181860F2C
:104A9000971F9583848382819381840F951F9783C9
:104AA00086832F7E25A3089580859185860F971F85
:104AB0009583848382859385840F951F978386834E
:104AC0000895FC012481358180819181A901481BD1
:104AD000590B57FF0DC03587248788279927841BDA
:104AE000950B958B848B21503040280F391F09C0BE
:104AF00095878487558B448B9C0121503040240F2F
:104B0000351F318B208B08950F931F938C01D9DFB4
:104B1000C8010296D6DF1F910F910895CF92DF92C0
:104B2000EF92FF920F931F937C01690181DFF701E0
:104B300085A1806185A3C701B601A801A2DFC701D5
:104B4000E3DF1F910F91FF90EF90DF90CF900895DA
:104B500043985FDF439A08950F931F938C0168DF9A
:104B6000C801F6DF1F910F9108952F923F924F9247
:104B70005F926F927F928F929F92AF92BF92CF92ED
:104B8000DF92EF92FF920F931F93DF93CF93CDB7F6
:104B9000DEB72697DEBFCDBF9E838D832B013A0102
:104BA000890131E0232E312C201A310AC801880FE7
:104BB000991F22273327281B390B3A8329834398CF
:104BC000ED81FE8185A18F7E85A3A801460D571D2D
:104BD0008D819E814DDFA301401B510B8D819E81F4
:104BE000B20146DFB801640D751D8D819E81A30160
:104BF0003FDFB201601B710B8D819E81A30138DF05
:104C0000480121E030E03C832B83AA24BB2456C01A
:104C100037FC0AC008948108910889819A8102961C
:104C20009A838983280E391E0894A11CB11CEB813C
:104C3000FC813296FC83EB832E0E3F1E6501C40C73
:104C4000D51C8401060D171D8D819E81B601A8011A
:104C50000FDF7201EA18FB088D819E81B701A80160
:104C600007DF8301081919098D819E81B601A8010A
:104C7000FFDE8D819E81B701A801FADE6401C40CBC
:104C8000D51C8501060D171D8D819E81B601A801D9
:104C9000EFDE7201E818F9088D819E81B701A80145
:104CA000E7DE83010A191B098D819E81B601A801E7
:104CB000DFDE8D819E81B701A801DADEA814B90478
:104CC0000CF4A6CF439A2696DEBFCDBFCF91DF91DD
:104CD0001F910F91FF90EF90DF90CF90BF90AF901A
:104CE0009F908F907F906F905F904F903F902F900C
:104CF0000895CF93DF93EC0169DD882309F1CE019C
:104D0000029664DD8823E1F04398CE0160EF49DC30
:104D10006C897D894E895F898FA198A5FEDA888D7F
:104D2000998D9D878C878A8D9B8D9F878E878C8D93
:104D30009D8D998B888B8E8D9F8D9B8B8A8B439AB3
:104D4000DF91CF9108952F923F924F925F926F9291
:104D50007F928F929F92AF92BF92CF92DF92EF920B
:104D6000FF920F931F93DF93CF9300D000D0CDB766
:104D7000DEB72C013B015A0149011C830B83261726
:104D8000370714F44B0139018B819C818A159B05EF
:104D90002CF48B819C81BC82AB825C0114012618AF
:104DA000370894E02916310408F466C0EB81FC81D1
:104DB000EA19FB09FA83E983349708F45DC06301BB
:104DC0000894C11CD11C85010F5F1F4FC201B601A1
:104DD000A801C2DE7EEFE72E7FEFF72EE80CF91C6C
:104DE000C201B701A801B8DE0B811C81025010403E
:104DF000C201B601A801B0DEC201B701A801ACDE54
:104E000062E0E62EF12CE60CF71C5CEFC52E5FEF9E
:104E1000D52EC20CD31CC201B701A501960101E039
:104E200010E00E940F1C8B819C8101979C838B83D7
:104E3000C201B7014B815C8196010E940F1C42E0C8
:104E4000E42EF12CEA0CFB1CC980DA80ECEFFFEFBA
:104E5000CE0EDF1EC201B301A70121E030E08601C2
:104E60000E940F1C089481089108C201B401A70197
:104E700021E030E00E940F1C2496DEBFCDBFCF9111
:104E8000DF911F910F91FF90EF90DF90CF90BF9037
:104E9000AF909F908F907F906F905F904F903F90DA
:104EA0002F900895EF92FF920F931F937C01C901F9
:104EB000F801D70195960C9110E0017010709801DF
:104EC000261B370B280F391F041B150B0E0F1F1F36
:104ED000C70124DEC7010DDF1F910F91FF90EF90F6
:104EE00008952F923F924F925F926F927F928F928E
:104EF0009F92AF92BF92CF92DF92EF92FF920F9369
:104F00001F93DF93CF9300D000D0CDB7DEB71C0145
:104F10003B015C834B8359014801FA82E9822617E1
:104F2000370714F45B0139018B819C81881699063F
:104F30002CF4C4018B809C809C838B83F10185A120
:104F40008F7E85A3E980FA80E60CF71C89819A811F
:104F50008E0D9F1D8A159B056CF449805A808B81AC
:104F60009C81480E591E89819A81840D951D881552
:104F700099053CF0C101B3014B815C81950184012D
:104F800022C06401E981FA81CE1ADF0AC101B301AE
:104F90004B815C819701860185DFC101B7014B819F
:104FA0005C81950182017EDF750189819A81E81A11
:104FB000F90AC101B701A2019501840173DFC101A2
:104FC000B301A60197016EDF2496DEBFCDBFCF915E
:104FD000DF911F910F91FF90EF90DF90CF90BF90E6
:104FE000AF909F908F907F906F905F904F903F9089
:104FF0002F900895CF92DF92EF92FF920F931F931D
:10500000CF93DF93EC013DDDCE017EDD6C897D89A0
:105010006115710579F48C859D85998B888B2DA1FF
:1050200030E0217030708A899B89820F931F9B8B9F
:105030008A8B13C04E895F8941155105C9F48E854D
:105040009F859B8B8A8B2DA130E0217030708889E1
:105050009989820F931F998B888BCE014ADE8C81B0
:105060009D81998388838E819F819B838A8357C08A
:105070002C813D81888199812817390724F0A1E08E
:10508000CA2ED12C03C0CC24CA94DC2C2E813F81A3
:105090008A819B812817390724F0F1E0EF2EF12C4B
:1050A00003C0EE24EA94FE2C8B01041B150B4398DD
:1050B00022C0CE01AEDCA801440F551F2E893F89C6
:1050C000CA01820F931F1816190644F4021B130B12
:1050D000888199818C0D9D1D998388838C899D89F8
:1050E0004817590744F4080F191F8A819B818E0DB8
:1050F0009F1D9B838A83288139818C819D812817FC
:105100003907B9F62A813B818E819F81281739079B
:1051100081F68DA180FF02C0CE017BDC439ADF9136
:10512000CF911F910F91FF90EF90DF90CF90089556
:105130002F923F924F925F926F927F928F929F92A7
:10514000AF92BF92CF92DF92EF92FF920F931F9395
:10515000DF93CF93CDB7DEB72697DEBFCDBF9C835D
:105160008B832B015E834D83A901380126173707F6
:1051700014F4AB0129018D819E81681679062CF407
:10518000C3016D807E809E838D83FA01E419F50949
:10519000FA83E983E430F10508F45EC013018D81E0
:1051A0009E81281A390A94E02916310408F454C063
:1051B00012E0A12EB12CA40CB51C4F01ECEFFFEFB7
:1051C0008E0E9F1E8B819C81B5014D815E81940165
:1051D00001E010E00E940F1C72010894E11CF11C18
:1051E000C980DA808EEF9FEFC80ED91EED81FE8157
:1051F0003196FE83ED838B819C81B701AF019601CF
:105200000E940F1C8D819E8101969E838D83ECEF01
:10521000FFEF2E0E3F1E8B819C81B2014D815E817E
:1052200029813A8181010E940F1C8EEF9FEF680E49
:10523000791E8B819C81B701A301960101E010E0EA
:105240000E940F1C0894611C711C8B819C81B5010C
:10525000A30194010E940F1C2696DEBFCDBFCF9103
:10526000DF911F910F91FF90EF90DF90CF90BF9053
:10527000AF909F908F907F906F905F904F903F90F6
:105280002F9008952F923F924F925F926F927F924C
:105290008F929F92AF92BF92CF92DF92EF92FF9246
:1052A0000F931F93DF93CF9300D000D0CDB7DEB71D
:1052B0003C017A836983FC0185A18F7E85A3AA24A2
:1052C000BB24A21AB30A229F1001239F300C329FE5
:1052D000300C11242501440E551E4A018A189B08E2
:1052E000BC82AB8235C0229FC001239F900D329FAC
:1052F000900D1124840F951F28163906CCF0E980F3
:10530000FA80E20EF31E220F331FCC24DD24C21AD2
:10531000D30AC301B701A201960101E010E00E9487
:105320000F1CC301B701A40196010E940F1C05C008
:105330002F5F3F4F12161306B4F68B819C810196A6
:105340009C838B830894411C511C0894810891080C
:10535000EB81FC811E161F064CF0EE9FA001EF9F13
:10536000500DFE9F500D11249501E4CF2496DEBF11
:10537000CDBFCF91DF911F910F91FF90EF90DF9004
:10538000CF90BF90AF909F908F907F906F905F90E5
:105390004F903F902F9008950F931F93FC018B0126
:1053A0004398808D918D95878487828D938D978783
:1053B0008687848D958D918B808B868D978D938B31
:1053C000828BCF0160EFEDD8C80160EF70E040E460
:1053D00051E00E948D21439A1F910F9108959C01E5
:1053E000813891059CF084EB91E0FC01459154914A
:1053F0004217530721F0452B49F00296F6CF00974C
:1054000029F09C01245B304035952795C90108950A
:105410007F928F929F92AF92BF92CF92DF92EF9244
:10542000FF920F931F93CF93DF938C01FC0185A113
:1054300082FF43C06A30710509F03FC084A1982FF4
:105440009695969596959827892F8295869586703C
:105450008927482F80FF18C0828593859383828394
:1054600086A52081318141FF06C0992787FD90954F
:10547000281B390B06C0992787FD9095280F391FE7
:10548000F80131832083D2C0F80180859185918312
:10549000808386A52281338142FF06C0992787FD3C
:1054A0009095281B390B06C0992787FD9095280FEA
:1054B000391FF80133832283B9C0CB0190DF9C01EF
:1054C000F80147A550A9841795073CF081A992A936
:1054D000840F951F2817390714F02FE330E0490196
:1054E000841A950AF80165A576A4E3A4F4A4161617
:1054F0000CF455C0A1A8B2A8603FD9F4C0E0D0E038
:10550000CC24DD2480E020E030E00EC0F70194914F
:105510002815390511F4892F6E010894E11CF11C3E
:10552000C90FD11D2F5F3F4F2A153B057CF3682F14
:105530005DC0C0E0D0E0CC24DD2430E042E050E0AB
:10554000A1E0B0E0F7010894E11CF11C7491272F51
:105550002F70261BCA0102978815990511F4322F66
:105560006E01C20FD11DAA15BB0599F0872F90E0DF
:1055700074E0959587957A95E1F78F70861BA8154D
:10558000B90511F4382F6E01C80FD11D4A155B05FE
:1055900011F4632F2BC04E5F5F4F1296D3CFC62FEF
:1055A000DD27C7FDD0952796C87F8C2F90E023E09C
:1055B000959587952A95E1F7272D332727FD309577
:1055C000A901849F9001859F300D949F300D112477
:1055D000882D90E0FC012E9FC0012F9F900D3E9FD3
:1055E000900D1124E80EF91ECC24DD24F80184A1CD
:1055F000982F83FF03C0872D762E682F94FD619529
:1056000095FD7194F80185A1806185A3772767FDD9
:105610007095472D552747FD5095C80132DAC801CE
:1056200073DAC801B701AE019601FAD8DF91CF91C4
:105630001F910F91FF90EF90DF90CF90BF90AF90B0
:105640009F908F907F900895FC0186A1282F30E0D5
:10565000C9018F709070892B01F121FF02C07595EF
:10566000679584A183FF0CC02281338185FF03C02D
:10567000260F371F02C0261B370B33832283089562
:105680002081318184FF05C0260F371F318320839D
:105690000895261B370B318320830895DC01FB011D
:1056A0009D968C919D97482F552747FD5095141630
:1056B0001506ACF19F966D917C91D097E617F70790
:1056C00054F09F01260F371FD1968D919C91D29750
:1056D0002817390714F0EFE3F0E09F01261B370B82
:1056E0009B96ED91FC919C978FEF403F580731F4CA
:1056F000E20FF31F8491482F50E011C0C901959526
:105700008795E80FF91F849120FF02C082958F7062
:1057100090E08F7090709C01241B350BA901CA0189
:105720000895EF92FF920F931F93DF93CF9300D0D2
:10573000CDB7DEB77C017A83698300E010E0CE014B
:1057400001960E943622BC01009729F0C701A6DF0E
:10575000080F191FF4CFC8010F900F90CF91DF9160
:105760001F910F91FF90EF9008950F931F93DF9378
:10577000CF9300D0CDB7DEB78C017A836983FC016B
:1057800086A190E08F709070892B19F460E070E032
:1057900005C069817A81C801C4DFBC01C80154DF3A
:1057A000CE0101960E943622BC01009719F0C80173
:1057B0002FDEF6CF0F900F90CF91DF911F910F91B9
:1057C0000895EF92FF920F931F93DF93CF9300D032
:1057D000CDB7DEB77C017A83698300E010E0CE01AB
:1057E00001960E947A22BC01009729F0C70156DF7A
:1057F000080F191FF4CFC8010F900F90CF91DF91C0
:105800001F910F91FF90EF9008950F931F93DF93D7
:10581000CF9300D0CDB7DEB78C017A836983FC01CA
:1058200086A190E08F709070892B19F460E070E091
:1058300005C069817A81C801C4DFBC01C80104DFE9
:10584000CE0101960E947A22BC01009719F0C8018E
:10585000DFDDF6CF0F900F90CF91DF911F910F9169
:105860000895DC01FB01CB010196E4919D96EC9338
:105870009D979C012F5F3F4FFC0184919E968C93D6
:105880009E97C9010196F90124919F962C939F97A9
:10589000D0961C92D097FC012491D1962C93D1974D
:1058A000D2961C92D29701969C969C938E939B972E
:1058B000089518951895EDE6F0E080818068808362
:1058C0000895579880E88BB939984198429882E0BA
:1058D0008A95F1F789B19AB1906C9AB998B19660AE
:1058E00098B997B1966097B98095881F8827881FC7
:1058F00008958FE980937A00662341F057985F9866
:105900004298399841985E9A81E407C05F983A9826
:105910004298419A56985E9882E480937C0082E097
:105920008A95F1F78FED80937A00889580917A00BF
:1059300086FDFBCF209178003091790010927A009B
:105940008AB1806C8AB988B1866088B987B186606F
:1059500087B9C9010895579880E88BB9399841985B
:10596000429882E08A95F1F74F9B0CC084E08BBB94
:1059700090916800809168008460809368008895A9
:10598000909368008AB1806C8AB988B1866088B9C2
:1059900087B1866087B980E008956F927F928F9279
:1059A0009F92AF92BF92CF92DF92EF92FF920F93AE
:1059B0001F933B015A0149017801E21AF30A0027BB
:1059C000F7FC0095102F9C01261B370B442737FD51
:1059D0004095542FC801B7010E94533CA618B70840
:1059E000CC24B7FCC094DC2CA60195010E949E3CFF
:1059F000820E931EC4011F910F91FF90EF90DF90D4
:105A0000CF90BF90AF909F908F907F906F900895B0
:105A10000F931F93CF93DF9360916403617083E7CB
:105A200093E067DF9C0160913A0470913B044091E0
:105A30003E0450913F048091640390E0EC01C170FA
:105A4000D07080FF03C000E411E002C000EF10E05E
:105A5000C90120E030E0A1DF909343048093420429
:105A600060E0CD2B09F461E083E793E042DF9C0125
:105A700060913C0470913D04409140045091410478
:105A80008091640380FD03C000E411E002C000EFD8
:105A900010E0C90120E030E080DF9093450480935E
:105AA0004404DF91CF911F910F9108959091640369
:105AB000492F50E09A0135952795822780FD03C034
:105AC00064E170E009C040FD03C060EF70E002C017
:105AD00060E471E06451704081FD03C044E150E036
:105AE00009C040FD03C040E451E002C040EF50E077
:105AF0004451504080E493E024E130E0C3CBCF93A5
:105B0000DF93EC0183E793E0DCDE882359F42197EF
:105B100051F088EE93E0E0E9F1E03197F1F7019779
:105B2000D1F7F0CF81E0DF91CF910895CF92DF924E
:105B3000EF92FF920F931F93CF93DF9380E493E054
:105B400060E070EE40E050EE20E030E200E010E275
:105B50000E9436238AE290E06AE270E00E94331CE1
:105B60008091640390E09C012170307080FD03C03F
:105B700060EF70E002C060E471E0EB01D595C7957D
:105B8000232B19F440E451E002C040EF50E07A01C9
:105B9000F594E79480E493E0BE0140E050E00E9479
:105BA000182580E493E06EE975E32FDE40916E03E3
:105BB000552747FD509580E493E0BE010E941825CB
:105BC00080E493E062E975E320DE89E59EEC909342
:105BD00068038093670380E493E062E070E04AE248
:105BE00050E00E94182580916503806180936503D1
:105BF00080E493E06CEE70E04CEE50E00E944125B2
:105C000080E493E00E94612582E493E00E94612594
:105C100080E493E06ED880E098EF909368038093DF
:105C2000670310E0812F42DF1F5F1430D9F780E453
:105C300093E06AEA75E115DE82E0809366038FE106
:105C400090E0909368038093670389E59EEC9093BE
:105C50006A0380936903809165038D7F8093650358
:105C600080916E03992787FD9095A701481B590BDA
:105C700080E493E0BE010E94182580E493E06BE786
:105C800075E3C3DD80E493E0BE01A7010E941825FF
:105C900080E493E066E675E3B8DD80EE97E09093EC
:105CA000680380936703FF248CE291E028DF882358
:105CB00009F4E2C060916403617083E793E019DE48
:105CC0008C01609164036095617083E793E011DE5D
:105CD00021E00038120714F460E006C022E000382A
:105CE00012070CF4C9C061E0AC0181E040385807EC
:105CF00034F022E0403852070CF4BEC06260262F18
:105D000030E0F901EE0FFF1FEE0FFF1FEA5BFB4FC4
:105D100011830083F901EE0FFF1FEE0FFF1FE85BF9
:105D2000FB4F5183408381E090E0062E02C0880F34
:105D3000991F0A94E2F7182F90E02F2D30E082236C
:105D40009323892B19F4862FB1DEF12A88EE93E094
:105D5000E0E9F1E03197F1F70197D1F78FE0F8161C
:105D600009F0A2CF00914E0410914F048091460497
:105D700090914704080F191F15950795E09052045C
:105D8000F090530480914A0490914B04E80EF91E60
:105D9000F594E7948091640390E041E0C42ED12C07
:105DA000C822D92280FD03C0C0EFD0E002C0C0E409
:105DB000D1E0B701601B710B882777FD8095982F84
:105DC00024E130E040E050E00E94533CA8979E015F
:105DD000442737FD4095542F0E949E3C021B130B15
:105DE00010933B0400933A042E0D3F1D30933F0463
:105DF00020933E0400914C0410914D04809148047E
:105E000090914904080F191F15950795E0905404C7
:105E1000F09055048091500490915104E80EF91EC1
:105E2000F594E794CD2819F4C0E4D1E002C0C0EFA6
:105E3000D0E0B701601B710B882777FD8095982F04
:105E400024E130E040E050E00E94533CA8979E01DE
:105E5000442737FD4095542F0E949E3C021B130B94
:105E600010933D0400933C042E0D3F1D30934104DC
:105E70002093400481E001C080E0DF91CF911F9129
:105E80000F91FF90EF90DF90CF900895FC018181FA
:105E90006281833024F4A82FA65F615002C0A82F2E
:105EA000A250772767FD70954381552747FD509590
:105EB0002081332727FD3095225F3F4FCA019595FA
:105EC000879595958795280F391F440F551F241BDB
:105ED000350B260F371F7595679575956795260FB6
:105EE000371F83EFA802C00111248095909565E0CB
:105EF00070E00E948B3CC901860F971F67E070E03D
:105F00000C948B3CFC012181223061F48281992721
:105F100087FD909583709070892B11F48DE1089521
:105F20008CE10895332727FD3095C901F3E095955D
:105F30008795FA95E1F78227932780FD02C08EE1CD
:105F400008958FE10895FC0181818F5F81838D30F9
:105F50002CF081E0818382818F5F828308951F937B
:105F6000CF93DF93EC0118811F5F1883CBDF81177C
:105F700024F481E08883CE01E6DFDF91CF911F9189
:105F80000895FC01818181508183882329F48281D5
:105F9000815082838CE081830895CF93DF93EC015D
:105FA000888181508883882329F4CE01EADFCE01DD
:105FB000A9DF8883DF91CF910895FC0190818091C2
:105FC0001601981791F4918180911701981769F43F
:105FD000928180911801981741F420E0938180917B
:105FE0001901981719F421E001C020E0822F0895CB
:105FF000A0915604B09157046091420470914304FB
:106000004091440450914504EFE5F4E020E030E095
:1060100017C080819181681779077CF08481958110
:106020006817790754F482819381481759072CF037
:10603000868197814817590744F02F5F3F4F389664
:106040002A173B0734F32FEF3FEFC901089585E28C
:10605000809313018BE18093140181E080931501FB
:1060600089E08093160182E08093170181E180939B
:10607000180108950F931F9360E070EE40E050EE1A
:1060800020E030E200E010E20E9436231F910F91E1
:106090000895EF92FF920F931F938C017B01BA0139
:1060A000A9010E941825C801B701AFDB1F910F910C
:1060B000FF90EF9008952F923F924F925F926F92D0
:1060C0007F928F929F92AF92BF92CF92DF92EF9288
:1060D000FF920F931F93DF93CF93CDB7DEB72E9729
:1060E000DEBFCDBF2C017E876D8758874F831A870F
:1060F0000987FC86EB8637FF05C080E493E0BA0190
:1061000010DB9C0186EF9FEF480E591EC901959543
:1061100087957201E81AF90AAAE0B0E04A0E5B1E00
:1061200044E1C42ED12CC20ED31ECE0CDF1C2EEFA8
:10613000A22E2FEFB22EED85FE85AE0EBF1E99E189
:10614000892E912C8E0E9F1E88E1682E86EC782E6B
:10615000709268036092670380E493E0B701A50141
:10616000960184010E94522729853A85309368035D
:1061700020936703C70102979E838D83D5011297F1
:10618000BC83AB830BE1202E312CED85FE852E0EDA
:106190003F1E80E493E06D817E81AD019701810116
:1061A0000E94522796012E5F3F4F3A83298380E455
:1061B00093E0B7014B815C8185010E9452278B855A
:1061C0009C85909368038093670380E493E0B60115
:1061D000A50129813A8181010E94522780E493E040
:1061E000B701A40196010E9452270894E108F10822
:1061F0004D855E85465E5F4F80E493E0B7010E9467
:10620000182580E493E00E94A8250894C11CD11CA5
:106210004D855E854350504080E493E0B6010E9476
:10622000182580E493E00E94A82580E493E0B20161
:106230004D855E850E9418251092680310926703B1
:1062400070926A0360926903809165038D7F8093E9
:10625000650380E493E06F81788587DAA985BA8544
:10626000EB85FC85AE17BF0741F1E0915604F09134
:1062700057043196F0935704E0935604319713E096
:10628000EE0FFF1F1A95E1F7CF01815A9B4F2D8129
:106290003E81DC012D933C93AF014F595B4F2B8125
:1062A0003C81DA012D933C93ED59FB4FA981BA81D2
:1062B000B183A083FC01378226822E96DEBFCDBF3C
:1062C000CF91DF911F910F91FF90EF90DF90CF90D2
:1062D000BF90AF909F908F907F906F905F904F9006
:1062E0003F902F900895CF92DF92EF92FF920F93FD
:1062F0001F93C0904203D090430320914A033091F2
:106300004B03C21AD30A00D000D000D0EDB7FEB7BD
:1063100031960FEC14E0ADB7BEB712961C930E93F6
:1063200011972DED35E33383228395838483F3D74F
:106330008DB79EB706969EBF8DBF8CE890E0B601E4
:10634000A80120E530E00FE110E0FFE1EF2EF12C95
:10635000B2DE8CE390E0B60140E051E02FEF3FEF7A
:106360000EE917EFE0E1EE2EE4E8FE2EA4DE8CED60
:1063700090E0B60144E051E02FEF3FEF9CDE1F912B
:106380000F91FF90EF90DF90CF900895DF92EF9202
:10639000FF920F931F93D82E87FF6CC083E190E08C
:1063A00062E070E00E94331C80E493E067EC75E3E8
:1063B00048E750E020E030E06CDEB9E5EB2EBEECC3
:1063C000FB2EF0926803E092670380E493E062E0C2
:1063D00070E043E150E02CEE30E00BE211E00E946F
:1063E0008E2580E493E00E94792610926803109233
:1063F0006703F0926A03E0926903809165038D7FE1
:10640000809365031092660380E493E062EC75E389
:1064100041E050E022E230E03CDE80E493E06DEBCE
:1064200075E341E050E028E430E033DE80E493E0BF
:1064300069EB75E341E050E02EE630E02ADE80E4CF
:1064400093E064EB75E341E050E024E930E021DEC5
:1064500080E493E06FEA75E341E050E02AEB30E03E
:1064600018DE80E493E06AEA75E341E050E020EE54
:1064700030E00FDE80E493E06AEA75E1F2D982E071
:106480008093660380E493E068E770E04EE150E0BB
:106490000E94182510925704109256041D2DD0FE0C
:1064A0000EC080915E0424E68202C0011124209176
:1064B0005D04332727FD3095820F931F14DF88E793
:1064C00090E066E270E00E94A91B11FF06C0809177
:1064D0005C04992787FD909506DF88E790E066E2E7
:1064E00070E00E94A91B12FF06C080915B049927EF
:1064F00087FD9095F8DE88E790E066E270E00E9404
:10650000A91B13FF06C080915A04992787FD909517
:10651000EADE88E790E066E270E00E94A91B14FFC3
:1065200006C080915904992787FD9095DCDE88E7A5
:1065300090E066E270E00E94A91B15FF06C0809102
:106540005804992787FD9095CEDE88E790E066E2B3
:1065500070E00E94A91BD7FE18C088E290E064E0BA
:1065600071E046E051E02FEF3FEF0EE917EFA0E1B9
:10657000EA2EA4E8FA2E9FDD80EA90E064E071E064
:1065800049E051E02FEF3FEF96DD1F910F91FF9013
:10659000EF90DF900895CF92DF92EF92FF920F93EA
:1065A0001F93CF93DF93A8E5B4E0E3E1F1E087E048
:1065B00001900D928150E1F780E493E05BDD8FEF75
:1065C000E5DE109249031092480310924B0310929B
:1065D0004A0380E493E04EDD88E592E090DA882378
:1065E00009F47AC180EE9FEF90936803809367036C
:1065F000CC24DD24EE24FF240FE311E0CFEED0E025
:1066000078C006DA80E89FEF909368038093670371
:1066100060914204709143044091440450914504B8
:1066200080E493E024E130E00E9442298FE190E091
:1066300090936803809367036091420470914304D0
:10664000409144045091450480E493E024E130E01B
:106650000E94B52560914204709143044091440426
:106660005091450480E493E025E130E00E94B52597
:106670006091420470914304409144045091450458
:1066800080E493E026E130E00E94B5254091420489
:1066900050914304CA014597C817D90714F0EA017D
:1066A00066972091440430914504C9014597081725
:1066B00019071CF0890106511040CA0145968E1534
:1066C0009F052CF096E1E92EF12CE40EF51EC90190
:1066D00045968C159D052CF086E1C82ED12CC20E56
:1066E000D31E80ED97E0E0E9F1E03197F1F70197F3
:1066F000D1F783E793E0E5D8882309F082CF80E4DF
:1067000093E0BE01A801970186010E9436238FEF16
:106710003DDE80E493E0AEDC6BDCEC01863091057D
:1067200009F486C087309105BCF48230910509F4E4
:106730004EC0833091053CF4009759F181309105AA
:1067400009F03FCF34C08430910509F456C085303C
:1067500091050CF05EC045C08A30910509F492C0E5
:106760008B3091054CF48830910509F476C089305E
:1067700091050CF07DC067C08C30910509F497C07D
:106780008C3091050CF489C08D30910509F019CF3A
:10679000A3C080915D04815080935D0487FF92C007
:1067A00083E680935D0480915E0481500DC08091EA
:1067B0005D048F5F80935D0484360CF483C0109277
:1067C0005D0480915E048F5F80935E047BC0809146
:1067D0005C04815080935C0418160CF473C08CE048
:1067E00009C080915C048F5F80935C048D300CF451
:1067F00069C081E080935C0465C080915B04815036
:1068000080935B0418160CF45DC08BE594E07ADB92
:106810000CC010915B041F5F10935B048BE594E048
:1068200071DB81170CF04EC081E080935B044AC09D
:1068300080915A04815080935A0487FF43C087E1B6
:1068400080935A043FC080915A048F5F80935A040A
:106850008831C4F110925A0435C080915904815096
:106860008093590487FF2EC08BE3809359042AC07C
:10687000809159048F5F809359048C331CF11092DE
:10688000590420C08091580481508093580487FF98
:1068900019C08BE38093580415C0809158048F5F12
:1068A000809358048C3374F0109258040BC0A3E109
:1068B000B1E0E8E5F4E087E001900D928150E1F766
:1068C00081E00BC0D595C79581E090E002C0880FAC
:1068D000991FCA95E2F774CE80E0DF91CF911F91A6
:1068E0000F91FF90EF90DF90CF900895FC014181D0
:1068F0004150440F440F462B8081815090E0440F5B
:10690000440F9C0153E0359527955A95E1F7422BAA
:10691000EAE7F3E0E40FF11D8770907021E030E0CA
:1069200002C0220F331F8A95E2F7808182230895E7
:10693000FF920F931F93CF93DF93EC01FF2401E0AD
:1069400010E0CE01612FD2DF8111F02A1F5F1430D9
:1069500011F0000FF6CF8F2DDF91CF911F910F9186
:10696000FF9008951F93CF93DF93EC01162F8EDADB
:10697000E82F882309F44CC04881413039F48981DB
:10698000813009F445C0853081F442C0433011F0B4
:106990004F3121F489818A3041F43AC0493111F0F4
:1069A0004A3119F489818C3099F15981252F23506E
:1069B000253030F58FE12802C0011124840F2230E8
:1069C0000CF081508823E1F0282F332727FD3095E4
:1069D000612F772767FD7095CB010297281739073C
:1069E000B9F0CB0101962817390791F0CB018796B2
:1069F0002817390769F06E5C7F4F2617370741F07B
:106A0000E33041F45B3031F480E04051473018F41A
:106A100081E001C080E0DF91CF911F9108954F92F6
:106A20005F926F927F928F929F92AF92BF92CF921E
:106A3000DF92EF92FF920F931F93CF93DF934B015F
:106A4000B42EF1EFCF2EFFEFDF2EC80ED91EEB01D3
:106A5000219747FD03C089E59EEC02C080E098EFD6
:106A60009093680380936703B60161507040AE0154
:106A7000415050409601215E3F4F8E010B5E1F4FEB
:106A800080E493E0E1E0EE2EF12C0E94712780E893
:106A9000B81601F59601225E3F4F80E493E0B601FF
:106AA000AE0164968E010E94712789E59EEC909359
:106AB0006803809367039601235E3F4F219780E42C
:106AC00093E00894C11CD11CB601A4018E010E9460
:106AD00071278EC03FE0E32EEB2021F429E53EEC48
:106AE000FF2411C0EE2DF0E0E75DF94C4491842FB6
:106AF00090E083709070880F991F86599F4FFC011A
:106B000025913491F42E309368032093670382E03B
:106B1000A82EB12CAC0CBD1C02E1402E512C4C0E09
:106B20005D1E80E493E0B601AE01950182010E94F2
:106B30005227EE2081F0F694F694EF2DF0E0E3700A
:106B4000F070EE0FFF1FE659FF4F859194919093DF
:106B5000680380936703BEE16B2E712C6C0C7D1C67
:106B60008E010E5F1F4F80E493E0B501AE019301EB
:106B70000E945227EE2081F0F694F694EF2DF0E07B
:106B8000E370F070EE0FFF1FE659FF4F859194916F
:106B90009093680380936703ECE18E2E912C8C0C0C
:106BA0009D1C74E1A72EB12CAC0EBD1E80E493E0B9
:106BB000B401AE01930185010E945227EE2081F0BD
:106BC000F694F694EF2DF0E0E370F070EE0FFF1FF7
:106BD000E659FF4F859194919093680380936703E2
:106BE00080E493E0B601A201940185010E9452273E
:106BF000DF91CF911F910F91FF90EF90DF90CF9099
:106C0000BF90AF909F908F907F906F905F904F90CC
:106C100008958F929F92AF92BF92CF92DF92EF92A0
:106C2000FF921F93CF93DF93EC015B014A01122F78
:106C3000B9E0CB2ED12CC80ED91EA9E0EA2EF12C3A
:106C4000E60EF71E80E493E0B601A70129E030E0EC
:106C50000E94B525112341F080E493E0B601A7011D
:106C600025E030E00E944229669680E493E0BE0170
:106C7000A5010E94182580E493E0B4010E94052C30
:106C8000DF91CF911F91FF90EF90DF90CF90BF9059
:106C9000AF909F908F9008952F923F924F925F9266
:106CA0006F927F928F929F92AF92BF92CF92DF921C
:106CB000EF92FF920F931F93DF93CF93CDB7DEB781
:106CC0002897DEBFCDBF8091160190911701A0914A
:106CD0001801B091190189839A83AB83BC8380E446
:106CE00093E060E070EE40E050EE20E030E200E043
:106CF00010E20E94362383E190E062E070E00E949F
:106D0000331C80E493E068E770E040E050E00E94CC
:106D1000182580E493E06BE176E30E94052C88243B
:106D20003324992401C0882419E5C12E1EECD12EEC
:106D3000D0926803C092670380E493E062E070E061
:106D400043E150E02CEE30E00BE211E00E948E2592
:106D500080E493E00E947926109257041092560422
:106D60006A81772767FD7095615070408AE790E0EF
:106D70000E945A1E2DB73EB7285030403EBF2DBF4F
:106D8000EDB7FEB7319605ED14E0ADB7BEB712967C
:106D90001C930E93119721E136E33383228395836D
:106DA00084838B81992787FD909597838683B3D2BF
:106DB0002DB73EB7285F3F4F3EBF2DBF88E790E01D
:106DC0006EE170E0A80128E730E00FE110E0BFE1DC
:106DD000EB2EF12C70D984E190E06EE170E04AE195
:106DE00051E02FEF3FEF0EE917EFA0E1EA2EA4E804
:106DF000FA2E61D98CED90E06EE170E04CE151E04B
:106E00002FEF3FEF58D9882009F447C082EC90E07B
:106E10006AEF70E04EE151E02FEF3FEF4CD9109256
:106E20006603D0926A03C0926903809165038D7FE7
:106E30008093650320E0992009F421E08AE090E046
:106E400065EF70E04CE056E3E4DE20E031E09316BD
:106E500009F421E08AE090E063E171E047E056E365
:106E6000D8DE20E082E0981609F421E080E590E089
:106E700065EF70E042E056E3CCDE20E093E0991647
:106E800009F421E080E590E063E171E04CEF55E327
:106E9000C0DE82E08093660323C082E390E06AEF65
:106EA00070E046E251E02FEF3FEF0EE917EFF0E11F
:106EB000EF2EF4E8FF2EFFD8332019F44EE251E014
:106EC00002C046E351E084EB90E06AEF70E02FEF00
:106ED0003FEF0EE917EFE0E1EE2EE4E8FE2EEBD8EF
:106EE0008FE190E0909368038093670389E59EECBF
:106EF00090936A0380936903809165038D7F8093EB
:106F00006503DD24D39438E1E32EF12C6D2D772732
:106F100067FD709580EE95E30E945A1E00D000D068
:106F200000D0EDB7FEB7319605ED14E0ADB7BEB7B2
:106F300012961C930E93119729EF35E33383228326
:106F400095838483E8D12DB73EB72A5F3F4F3EBF7C
:106F50002DBF80E493E0B7014CE350E00E94182578
:106F600080E493E0B8010E94B52BD39437E0D316A8
:106F700009F4DD2480E290E0E80EF91E98EFE916AE
:106F8000F10421F6109268031092670380E493E005
:106F900068E070E040E550E028EE30E001E510E008
:106FA0000E9452273B81832F8B5F63E19BD4492F43
:106FB00083E19802C0011124885E6EE193D4292FE9
:106FC000842F6BE09BD4820F6DE18CD42B5E281B49
:106FD000832F859585953E5F830F67E083D4892F46
:106FE000820F87507FD4295FB22EB91A89819A8186
:106FF000AB81BC818D839E83AF83B88781E08D8315
:10700000CE0105960E94462F182F82300CF4195F8E
:10701000CE0105960E94CD2F11501130C9F74D8039
:107020005E806F80788481E090E0092C02C0880F38
:10703000991F0A94E2F7282E28E5C22ED12C70C0A1
:107040003E812A81321719F080E194E802C080E085
:1070500090E09093680380936703321761F4CE0148
:1070600005966B2D7FDC882331F080E098EF9093BC
:1070700068038093670300D000D000D0EDB7FEB75F
:10708000319605ED14E0ADB7BEB712961C930E9382
:10709000119786EF95E3938382838D81992787FDEE
:1070A00090959583848337D12DB73EB72A5F3F4FA4
:1070B0003EBF2DBF80E493E0B701A6010E941825D2
:1070C00080E493E0B8010E94B52B9E818A819817D5
:1070D00091F4CE0105962CDC182F81101221CE01DF
:1070E00005960E94DD2F81111068112321F0C70140
:1070F000B601412F94DCCE0105960E94AF2F80E2AD
:1071000090E0E80EF91E98EFE916F10409F098CF27
:10711000A8E1B0E0CA0EDB1EB8EECB16D10461F0D8
:1071200098E1E92EF12C8CCF88EE93E0E0E9F1E0D4
:107130003197F1F70197D1F783E793E00E94612C33
:10714000882391F788E592E00E947F2D882309F437
:10715000BFC00E94082D0E94F82F8130910589F050
:10716000823091051CF4892B39F013C082309105CF
:1071700069F0039771F4ADC0CE0101960E94C12F52
:10718000D3CDCE0101960E94A32FCECD81E08826DB
:10719000CBCD882089F22091440430914504C90167
:1071A000805F9040CC9788F499242E50314014F0A1
:1071B00099249394809142049091430480359105E1
:1071C0000CF4B2CD92E0992AAFCD4D825E826F82EF
:1071D000788688E5A82EB12C77C0209142043091A2
:1071E0004304C6014097281739070CF457C0C6015D
:1071F0000F96821793070CF451C0209144043091EC
:107200004504C5010397281739070CF447C0C50189
:107210004496821793070CF441C0EE818A81E817E7
:1072200009F03CC0E150EE0FEE0FE9298D8181504D
:1072300090E0EE0FEE0F9C0103E0359527950A953F
:10724000E1F7E22BF0E0E658FC4F8770907021E008
:1072500030E002C0220F331F8A95E2F78081822737
:1072600080838E010B5F1F4FC80162DBF82EF22076
:10727000C8010E94DD2F882311F0A0E8FA2AC60178
:10728000B5014F2DCCDB88EE93E0E0E9F1E03197DA
:10729000F1F70197D1F7332433944ECFCE01059601
:1072A0000E94AF2F20E230E0C20ED31E38EFC3168B
:1072B000D10409F092CF88E190E0A80EB91E98EEB3
:1072C000A916B10409F42FCD18E1C12ED12C85CF18
:1072D0003324832D2896DEBFCDBFCF91DF911F9140
:1072E0000F91FF90EF90DF90CF90BF90AF909F9065
:1072F0008F907F906F905F904F903F902F90089568
:10730000F894AAC3FC0105900020E9F780959095B8
:107310008E0F9F1F0895AEE0B0E0E0E9F9E337C3B8
:107320000D891E898EE08C831A8309838FEF9FE776
:107330009E838D839E01275E3F4FCE0101966F890C
:10734000788DA90109D02F813885020F131FF8010C
:1073500010822E96E4E037C3ABE0B0E0E1EBF9E356
:1073600008C33C012B015A01FC011782168283815C
:1073700081FD03C06FEF7FEFB9C19AE0892E1E0136
:107380000894211C311CF3012381F20123FD859116
:1073900023FF81912F01882309F4A5C1853239F497
:1073A00023FD859123FF81912F01853221F490E007
:1073B000B301EFD1E8CF982FFF24EE249924FFE109
:1073C000FF15D0F09B3269F09C3228F4903259F0CE
:1073D000933291F40EC09D3249F0903369F441E04C
:1073E00024C052E0F52A84E0F82A28C098E0F92A5F
:1073F00025C0E0E1FE2A22C0F7FC29C0892F805376
:107400008A3070F4F6FE05C0989C902C1124980EDA
:1074100015C0E89CE02C1124E80EF0E2FF2A0EC013
:107420009E3229F4F6FC5FC140E4F42A07C09C3682
:1074300019F450E8F52A02C0983649F4F20123FD08
:10744000959123FF91912F01992309F0B8CF892FAE
:107450008554833018F08052833038F444E050E093
:10746000A40EB51E5FE359830FC0933631F09337F6
:1074700079F0933509F052C01FC0F50180818983EE
:1074800042E050E0A40EB51E610101E010E011C021
:10749000F501C080D180F6FC03C06FEF7FEF02C022
:1074A000692D70E042E050E0A40EB51EC60166D121
:1074B0008C015FE7F52213C0F501C080D180F6FC96
:1074C00003C06FEF7FEF02C0692D70E042E050E033
:1074D000A40EB51EC60147D18C0150E8F52AF3FE73
:1074E00006C018C080E290E0B30153D1EA948E2D1B
:1074F00090E008171907B0F30DC0F601F7FC85916D
:10750000F7FE81916F0190E0B30143D1E110EA945D
:10751000015010400115110581F7E2C0943611F0B9
:10752000993661F5F7FE08C0F5012081318142816D
:10753000538184E090E00AC0F501808191819C0133
:10754000442737FD4095542F82E090E0A80EB91EE5
:107550009FE6F92257FF09C0509540953095219537
:107560003F4F4F4F5F4FE0E8FE2ACA01B901A1012A
:107570002AE030E03AD1D82ED2183FC0953729F40E
:107580001F2D1F7E2AE030E01DC01F2D197F9F3662
:1075900061F0903720F4983509F0A5C00FC09037FE
:1075A00039F0983709F09FC004C028E030E00AC0E5
:1075B000106114FD146020E130E004C014FD166079
:1075C00020E132E017FF08C0F501608171818281FE
:1075D000938144E050E008C0F50180819181BC01B5
:1075E00080E090E042E050E0A40EB51EA101FDD085
:1075F000D82ED2188FE7F82EF122F6FE0BC05EEFE0
:10760000F522D91438F4F4FE07C0F2FC05C08FEE61
:10761000F82202C01D2D01C0192DF4FE0DC0FE017F
:10762000ED0DF11D8081803319F499EEF92208C027
:107630001F5FF2FE05C003C08F2D867809F01F5F23
:107640000F2DF3FC13C0F0FE0EC01E1510F09D2C84
:107650000AC09D2C9E0C911A1E2D05C080E290E060
:10766000B30197D01F5F1E15C8F304C01E1510F498
:10767000E11A01C0EE2404FF0EC080E390E0B301E4
:1076800088D002FF1BC001FD03C088E790E00EC058
:1076900088E590E00BC0802F867881F001FF02C062
:1076A0008BE201C080E2F7FC8DE290E0B30171D083
:1076B00005C080E390E0B3016CD09A94D914C8F36C
:1076C000DA94F101ED0DF11D808190E0B30161D0FC
:1076D000DD20B1F705C080E290E0B3015AD0EA9412
:1076E000EE20C9F750CEF30166817781CB012B964E
:1076F000E2E15BC1DC01CB01FC01F999FECF06C0E0
:10770000F2BDE1BDF89A319600B40D92415050405F
:10771000B8F70895F999FECF92BD81BDF89A9927DF
:1077200080B50895DC01A40FB51F4150504040F0D2
:10773000CB01840F951F2E9105D041505040D8F7B2
:107740000895262FF999FECF92BD81BDF89A019731
:1077500000B4021639F01FBA20BD0FB6F894FA9A99
:10776000F99A0FBE0895FC01059061507040011018
:10777000D8F7809590958E0F9F1F0895FC0161505A
:10778000704001900110D8F7809590958E0F9F1F43
:1077900008950F931F93CF93DF938C01EB018B819F
:1077A00081FF1BC082FF0DC02E813F818C819D8196
:1077B0002817390764F4E881F9810193F983E88394
:1077C00006C0E885F985802F0995892B31F48E81D3
:1077D0009F8101969F838E8302C00FEF1FEFC80128
:1077E000DF91CF911F910F910895FA01AA272830B8
:1077F00051F1203181F1E8946F936E7F6E5F7F4F7E
:107800008F4F9F4FAF4FB1E03ED0B4E03CD0670FF9
:10781000781F891F9A1FA11D680F791F8A1F911D4C
:10782000A11D6A0F711D811D911DA11D20D009F49C
:1078300068943F912AE0269F11243019305D3193DE
:10784000DEF6CF010895462F4770405D4193B3E0C7
:107850000FD0C9F7F6CF462F4F70405D4A3318F06E
:10786000495D31FD4052419302D0A9F7EACFB4E01F
:10787000A6959795879577956795BA95C9F70097D7
:107880006105710508959B01AC010A2E0694579578
:10789000479537952795BA95C9F7620F731F841FCF
:1078A000951FA01D0895629FD001739FF001829FD4
:1078B000E00DF11D649FE00DF11D929FF00D839F7F
:1078C000F00D749FF00D659FF00D9927729FB00D1C
:1078D000E11DF91F639FB00DE11DF91FBD01CF012F
:1078E00011240895991B79E004C0991F961708F098
:1078F000961B881F7A95C9F78095089587FB082EF7
:10790000062687FD819567FD6195ECDF0EF4919564
:1079100007FC8195089597FB092E07260AD077FD6D
:1079200004D05ED006D000201AF4709561957F4F88
:107930000895F6F7909581959F4F089597FB092E2E
:1079400005260ED057FD04D05FD00AD0001C38F4B5
:1079500050954095309521953F4F4F4F5F4F08957B
:10796000F6F790958095709561957F4F8F4F9F4F5B
:1079700008952F923F924F925F926F927F928F92D3
:107980009F92AF92BF92CF92DF92EF92FF920F93AE
:107990001F93CF93DF93CDB7DEB7CA1BDB0B0FB6B8
:1079A000F894DEBF0FBECDBF09942A883988488875
:1079B0005F846E847D848C849B84AA84B984C8840B
:1079C000DF80EE80FD800C811B81AA81B981CE0F02
:1079D000D11D0FB6F894DEBF0FBECDBFED010895E7
:1079E000AA1BBB1B51E107C0AA1FBB1FA617B707E5
:1079F00010F0A61BB70B881F991F5A95A9F7809501
:107A00009095BC01CD010895A1E21A2EAA1BBB1BC3
:107A1000FD010DC0AA1FBB1FEE1FFF1FA217B3075A
:107A2000E407F50720F0A21BB30BE40BF50B661F70
:107A3000771F881F991F1A9469F760957095809534
:107A400090959B01AC01BD01CF010895EE0FFF1F82
:0C7A50000590F491E02D0994F894FFCF0C
:107A5C00E28093002B004F4B0041626272656368B9
:107A6C00656E00000000000000143C003E007A75BA
:107A7C0072C3BC636B00C3846E6465726E005A750E
:107A8C0072C3BC636B0053706569636865726E008A
:107A9C0000010202030303030404040404040404A9
:107AAC00050505050505050505050505050505057A
:107ABC00060606060606060606060606060606065A
:107ACC00060606060606060606060606060606064A
:107ADC00070707070707070707070707070707072A
:107AEC00070707070707070707070707070707071A
:107AFC00070707070707070707070707070707070A
:107B0C0007070707070707070707070707070707F9
:107B1C0008080808080808080808080808080808D9
:107B2C0008080808080808080808080808080808C9
:107B3C0008080808080808080808080808080808B9
:107B4C0008080808080808080808080808080808A9
:107B5C000808080808080808080808080808080899
:107B6C000808080808080808080808080808080889
:107B7C000808080808080808080808080808080879
:107B8C000808080808080808080808080808080869
:107B9C0000010102010202030102020302030304B9
:107BAC000102020302030304020303040304040599
:107BBC000102020302030304020303040304040589
:107BCC000203030403040405030404050405050669
:107BDC000102020302030304020303040304040569
:107BEC000203030403040405030404050405050649
:107BFC000203030403040405030404050405050639
:107C0C000304040504050506040505060506060718
:107C1C000102020302030304020303040304040528
:107C2C000203030403040405030404050405050608
:107C3C0002030304030404050304040504050506F8
:107C4C0003040405040505060405050605060607D8
:107C5C0002030304030404050304040504050506D8
:107C6C0003040405040505060405050605060607B8
:107C7C0003040405040505060405050605060607A8
:107C8C000405050605060607050606070607070888
:00000001FF
